:100000004D424E014D3448501102040001002200BF
:100010006000000000C000000000000000000000C0
:100020000000EEEE000000000000000000000000F4
:1000300001001102000000000000000000000000AC
:100040000200150100002B000000000000AC0000C1
:10005000030015012B00300000AC0000001400006C
:1000600000380020ED020000000000000000000049
:100070000000000000000000000000000000000080
:100080000000000000000000000000000000000070
:10009000000000000000000000000000B5010000AA
:1000A000E1010000FD010000B9010000CD010000E8
:1000B00000000000002934D00123002210B488423F
:1000C0002CD301242407A14204D2814202D2090187
:1000D0001B01F8E7E400A14204D2814202D24900A8
:1000E0005B00F8E7884201D3401A1A434C08A0424B
:1000F00002D3001B5C0822438C08A04202D3001BE1
:100100009C082243CC08A04202D3001BDC082243F7
:10011000002803D01B0901D00909E3E7101C10BC1B
:100120007047002801D00020C04307B4024802A154
:100130004018029003BDC046D90000000029F0D04D
:1001400003B5FFF7B9FF0EBC4243891A1847C046F2
:10015000002941D010B4041C4C40A44601230022C5
:10016000002900D54942002800D5404288422CD3BE
:1001700001242407A14204D2814202D209011B01B9
:10018000F8E7E400A14204D2814202D249005B00B8
:10019000F8E7884201D3401A1A434C08A04202D320
:1001A000001B5C0822438C08A04202D3001B9C0861
:1001B0002243CC08A04202D3001BDC0822430028C3
:1001C00003D01B0901D00909E3E7101C6446002C89
:1001D00000D5404210BC7047002806D003DB002049
:1001E000C043400801E08020000607B4024802A195
:1001F0004018029003BDC046190000000029EBD052
:1002000003B5FFF7A7FF0EBC4243891A1847C04643
:100210007047C046FEE70000034B01225A70A0233E
:100220000022DB051A707047000F0020034B0122EB
:100230009A70A0230022DB059A707047000F0020FF
:1002400008B5044B01221A70034B0022DA7700F044
:10025000A5FF08BD000F00200800005038B580251C
:10026000ED052B79DBB2002B0CD130490B604B60D4
:100270002B89081C9BB28B608A680C30103107F008
:10028000A5F847E0012B0DD1284BD968002941D0B2
:100290005A68186982423DDA5A68501C58602B7AB5
:1002A0008B5437E0022B30D1204CE368002B2AD04E
:1002B000226821698A420CDA22689B5C1BBAEB60D7
:1002C000A3682068C01880B207F0BEF82368013325
:1002D00017E0A2682368201C211CD2180C301031B2
:1002E00007F074F8E368002B0DD0A16822688A1823
:1002F000A2601B781BBAEB60A06880B207F0A4F87C
:100300000123236006E0EB6004E0032B02D1074BDE
:1003100000225A60C0468023DB0501221A70C046C5
:1003200002221A7000221A7038BDC0462003002035
:1003300080230222DB05FF321A600421024AFF31CA
:10034000118000221A70704706000040F8B5A02303
:10035000DB059B68494A1F21DBB21160D12B0BD012
:10036000D02B01D80133DBB2A022D2059168FF2047
:10037000814319439160F1E70023414A41499A18AA
:100380008A4204D24049C95804331160F5E73F4B13
:100390003F4A191D043B934203D200221A600B1CF2
:1003A000F6E7EFF308823B4B191D043B9A4203D951
:1003B000394818600B1CF7E7FFF7BAFF3749384890
:1003C000053904F00FFB374C374D01235B42237195
:1003D0006371A371E3712B1C3C331A782B1C3D33E2
:1003E0001B7880B21B02134398423FD106F0D6FF20
:1003F0002E4B2F4918882F4A88420BD06E7D1888C3
:100400002B7D36023343984204D113889BB223716B
:100410001B0A637113888B421BD0EE7DA87D138865
:1004200036023043834214D100200423013BDBB267
:10043000FF2B07D0204EEF18F65C3F79B742F5D17D
:100440000120F3E7002804D013889BB2A3711B0A94
:10045000E371637922791B0213438B4206D0E27960
:10046000A37912021A43124B9A4204D1134B02226F
:100470001A6062B6FEE701F0DFF9F7E728000050E6
:10048000000000202003002004A10000240300201D
:10049000FC0E00206C100020CDCDCDCD00C00000A2
:1004A00000000000040F0020C0BF0000FEAB0000F1
:1004B000FFFF0000BEBF000000AC000000E100E054
:1004C000014B18607047C0460C0F0020014B1868A4
:1004D0007047C0460C0F0020014B18607047C046A3
:1004E000100F0020014B18687047C046100F002005
:1004F000014B18687047C0460000002038B5154C05
:10050000256804F097FEA862256804F097FEE8626B
:10051000256804F097FE6861256804F097FEA861DD
:10052000256804F0ABFE2862256804F00FFFE8613F
:10053000256804F021FF084B08491B6809686862B8
:100540001878097C2268414302331161FC32136040
:1005500038BDC04600000020100F00200C0F002006
:1005600082B0F0B589B0109C151C0F9306930294CD
:1005700007900E1C119C04F0B3F947793A4B04978D
:100580008279964206D11B6800211A6AAB00D05AC4
:1005900003910BE01A68354B52691968731C89681E
:1005A00003964B43EB1801339B00D05A04997143D7
:1005B00049194A00A4182388069E0193019F7318C5
:1005C000874203D8C61B029FBE521CE0029EB6188B
:1005D00005960027F65F013610D01F787EB2B4462C
:1005E000013601DA013703E06646002E06DD013FE1
:1005F0001F7002235B42238001202FE0069F7918A1
:100600000F78002F01D120800CE07FB27C1C05D137
:10061000019E059F301A3880002002E0012F01D191
:10062000FF2008701978039C049E079F48B274430A
:100630007D19002805DC029EB25E013208D0002937
:1006400006D12A5700203E2A08DC0131197005E046
:100650002A57002A01DD01391970002009B0F0BCC9
:1006600008BC02B01847C046000000200C03002060
:10067000F0B58BB000AF04F033F906F031FF584C01
:100680006E4623689D68DB687D625A00111C0E313E
:100690009B00C9080E33C900DB08DB00761AB5469B
:1006A000F61A6D4600216846B546BD61FE6009F048
:1006B00031FA002004F03EFF7E6A4A4A206815683D
:1006C000B20052420368BA60321C5A439100F96189
:1006D000B107711A79609107891A3A62013B32D3E6
:1006E00044683E6A3219261C5E437618B400FE68E0
:1006F000920034197C61FC69A2420BD07C6904260B
:10070000A418A4466C697642A458B4446646346082
:10071000043AF0E7BE683A6AA419FC617C6A7E6814
:10072000121B3A628919D9E72F49F8697E23D2B2A0
:100730005B4208704A708A70CB7001205223BA69FC
:100740000B7106F0D1FD06F0A5FC0B2845D1002069
:1007500004F0F0FE224B1968224B08681C687B6A83
:10076000F86143439A003A629A07D21A3A617B6170
:10077000844666464A68013EB446D5D3654655432D
:100780007E691A48B31812185219BE6938695200A6
:10079000B2182D18FE68AD0075199B003D603E6AC9
:1007A000B3420ED03D68E818656904380668E85819
:1007B000301A0025565F864200DA1080043B023A68
:1007C000EDE7BD6876193E627D6A7E69761B7E61C3
:1007D0007D683E6976193E61CBE7BD460BB0F0BD42
:1007E0000C0300200000002048040020FFFFFF7FD2
:1007F00008B502F09BFC021E05D10749A9230B7125
:1008000006F072FDFEE7054B1B6803CB04F062F9AE
:10081000FFF774FE08BDC0464F0400200C03002003
:10082000114B01201B680022191C9431404210B565
:100830000A604861CA610C310A601C1C0B49B8345B
:100840002160A260283C6061181CAC302260103826
:1008500002618161191CBC31026024394A628C3307
:100860000A601A6010BDC04600000020FFFF0000B3
:10087000F0B585B000AFB960386005F017F88300B7
:100880000A33DB08DB00041C6846C01A854605F005
:1008900015F863000833DB08DB006E46F11A8D465D
:1008A0006D46281C7D6005F027F84C4B1B681A1C10
:1008B0009432106863280BDD012040428446181CE6
:1008C0000021A830654611601C38C5614162016095
:1008D0001168013111601A1C9032106863280DDD17
:1008E000012040428446181C0021A4301160654656
:1008F0008160191C05608C3101200860116801318C
:1009000011601A1CA0321068012808DD344D181C33
:100910000021B830116020380562816201601168E1
:1009200001311160191C9C310868012808DD002282
:100930002B480A600A621A1C8861983201211160F2
:100940001A1C9C321168013111600022111C013CFB
:1009500007D3A00030587D6809186000285A121883
:10096000F5E7181C0324013C002C19D0051CB035F8
:100970002E688E4200D22960051CA8352E688E4252
:1009800000D92960051CC0352E68964200D22A6025
:10099000051CB8352E68964200D92A600438E2E773
:1009A0001A1C8C3212683D6892009A18111CAC31E6
:1009B000A43209681268BE688A1A2A801A1C983202
:1009C0001268BD4692009B181A1CBC32B4331268E0
:1009D0001B68D31A338005B0F0BDC046000000206C
:1009E000FFFF0000F0B5234F1D1C3B68161CDA68A2
:1009F00085B0019192000021041C301C09F08AF896
:100A00003B68281C1A690021920009F083F8019FB5
:100A1000002F0CD0201C04F08DFD174B301C1B68E0
:100A2000291C5A691B6A06F065FE013FF0E7002C9D
:100A30000FD1114B1B685F69DB69029304F0E8FB7F
:100A4000039004F0EFFB0299031C039A381C06F094
:100A500065FD301C291C019A06F0F2FE002C06D11F
:100A6000054B201C1D6804F0C3FEFC35686005B012
:100A7000F0BDC0460C03002000000020F0B5161C9D
:100A800085B0902201900391081C5200002109F0CA
:100A900041F806F031FD0425013D2F4C002D2FD0EB
:100AA000019804F047FD23682C495A699F690A7030
:100AB0009A6804238A7001329200CB70B218A02386
:100AC00002204F700B7106F00FFC20684269571E20
:100AD000BC46E1D3836961465943039CC918890028
:100AE00061180439013B09D3846854431C1901344B
:100AF000A700BF590C68E7190F60F2E76246E6E706
:100B000027687C690294251CBC69013D0FD3261C13
:100B10006E43039A3619B6009619043E013CF3D38E
:100B200030680321FFF7C6FA00043060F5E70B4D8B
:100B3000029F1023AB71E4B204206023291C039AA6
:100B40002B712F706C70AC70E87006F0CDFB002339
:100B5000AB7105B0F0BDC0460C0300204804002076
:100B600030B52C4D85B02B681A1CE0321178683AEC
:100B7000002904D1191CC4310978002901D00021B1
:100B80001170117800291FD0DA6F234901929A6BF6
:100B9000002002921B6B01AA039303234B707C235A
:100BA0005B42CB7010230B7106F09EFB2B68002478
:100BB000191DDA6FC96F8A4202DC0132DA6725E05B
:100BC000DC67164B1C700FE01A1C79321478002C6D
:100BD0000CD0713A8833D06F1B68984203DC013027
:100BE000D0670C1C12E0D16701240FE09A6B1B6BDD
:100BF0000B49019202930920642301AA0B7103940B
:100C000006F072FB2B68DC670833DC67201C05B03C
:100C100030BDC046000000201C010020140F002041
:100C200023010020F0B591B004AFF9603A627B6116
:100C3000386106F061FCCB4B6D461B68BD611C68DA
:100C4000B86004346400221C0832D208D200AE1A04
:100C50005A68B54604325200131C0833DB08DB0027
:100C6000F61A04ADB5467D6204AD281C002108F0DB
:100C700051FF221C0021786A08F04CFFB86CBA4C76
:100C80000678236838695A69191CDB690090786A0C
:100C9000303104300190281D0290386A03F0C0F909
:100CA000B96C06430E70BE682368327B58690092A7
:100CB0007E6A191C019602956C3130333A6A03F052
:100CC0001BFBBD69BE6CAD4623683578FE681A6AA9
:100CD000191C5B6A00963031786903F017F9BE6C15
:100CE0000543357006F014FC051C06F07DFF2D79D8
:100CF000012D0AD1B4300368002B06D106F0E8F9C3
:100D0000012802D0281C03F0FDFF2568281C291C9F
:100D10006C31303003F0CAFA944A236812682867AD
:100D20000C20115EDD6D8D420EDC0E26915F186E7B
:100D3000884209DB1025515F5E6E8E4204DC122072
:100D4000125E9B6E934221DA00233B85282101230A
:100D5000CB5506F0CBF9002818D106F0A3F90028EE
:100D600014D0814B1A68FF239168FE2901DC936837
:100D7000DBB2381C292202212830D35506F052FA62
:100D80007B4804F05BFE03F0C3FEE2E7754D794952
:100D90002B6802241E6858689A68CB780E707F26EC
:100DA000B343802648708A707642386A2343013202
:100DB00033435200CB708218532301200B7106F08D
:100DC00093FA2B686C491B697F224B70CB7801200A
:100DD000934323433343CB707A696D230B7106F041
:100DE00083FA2B68282019682922C15558682A21BE
:100DF000D0559A682B20CA55591DC97F0132C1555B
:100E00001B692D202C21CB55C35D7F218B432343B0
:100E10001E43C3191E703E6A5200B2180092391C5C
:100E2000002201202831131C06F024FA02F000F9F8
:100E300002F04EF9FFF794FE002800D08DE04A4CF6
:100E40002368586904F052FC2368186F04F078FB9B
:100E500004F036F9BE6C3378002B71D12368396AFF
:100E60001A1C30321B68386906F0C0FB23687969A8
:100E70001A68F86806F00EFC06F02AF938620028B5
:100E80005ED16E4601207E6204F066FF2B68396AEF
:100E90009A695B695A435200131C0833DB08DB0074
:100EA000F01A854604AE301CFE6108F033FE06F0F1
:100EB0002FFB061C06F014FB296838614A69386A62
:100EC000246830607A607B68013B9C4629D38B693B
:100ED00062465A43F86C95004019FD69B8605000AD
:100EE0002818F860013B19D3BA68980010588D682B
:100EF000020C786845435D19A0690135AD002D5895
:100F0000501BFD685A00A8523D692D78A842E9DBC4
:100F100032680125101830603D62E3E762467A606E
:100F2000D1E73D6A002D06D10F4BF86C1B68F969BB
:100F30001A6806F0D3FD002004F00EFF7E6AB54665
:100F4000022003F00DFF786906F0EEFE064B1868EC
:100F5000743007F015FE002000E0201CBD460DB0E7
:100F6000F0BDC0460C03002000000020100F002040
:100F700010270000480400201C010020F0B5940058
:100F8000231C0A3385B0DB08DB006946C91A02AFAF
:100F90008D4602AA061C7A60101C0021221C08F053
:100FA000B9FD231C0833DB08DB006946C91A8D46EE
:100FB00002AD281C221C002108F0ACFD0C4C301C9A
:100FC0002368D96A9A6A6C3300910193291C7B6863
:100FD00007F0F8FD301C02F0DBF82368301C9A6A39
:100FE000DB6A291C00937B6807F032F8BD46F7BD29
:100FF0000000002070B50C1C151C1E1C07F080FAA8
:10100000144B201C1B68996ADA6A07F07FFB201CCE
:1010100007F08AFF201C07F075FC321C201C291CDD
:1010200007F02CFD201C291C02F0D8FE06F070FAF7
:10103000041C06F0D9FDA6300378002B09D12379D2
:10104000002B06D006F044F8012802D0012003F05E
:1010500059FE70BD0000002038B508F039FC051CB1
:10106000012008F049FC041C281C03F03FFC201C54
:1010700003F048FC38BD38B508F0E6FC08F030FC59
:10108000051C002008F038FC041C281C03F02EFC72
:10109000002004F0D5FA201C03F034FC03F014FE09
:1010A00038BD10B5A4B08C22041C002101A808F0A2
:1010B00031FD01A8211C07F01DFD07F045FD01A829
:1010C000211C02F0D5F824B010BD0000F8B506F0E0
:1010D0008BFD2E4DA6302B68007819794AB2002876
:1010E00001D1501C04D10024DC60FF335C7314E098
:1010F000DC682748844202DCDC680134DC60012AB9
:1011000004D0DE681F690124BE4200DA0C1CD968D5
:10111000814202DDFF330121597363B2934209D04A
:1011200000201C49231C0E33021C0B7106F0DCF856
:10113000286804712B681A79002A03D1164A1268AC
:10114000127804E0012A03D1134A126852781A6017
:10115000186804F04FFC2B68041CFC33586804F03A
:101160006DFC241A002C0BDD2B68186804F042FC7F
:101170002B68041CFC33586804F060FC201A00E063
:10118000012003F0BFFD03F0DFFDF8BD00000020EB
:101190002F7500004F040020100F002008B505F047
:1011A00097FF002802D1022004F09CF908BD00003E
:1011B000F0B589B0061C06F0ABF9059006F014FDF9
:1011C000031CB0331A68A14B002A08D1B83002685A
:1011D000511E8A41D2B20492002A06D001E00120B9
:1011E00004901A680021CC3205E01A68CC321168EC
:1011F000FE2901DC013111601B6800211A1CC83274
:1012000011700499002904D091490968097D0029C9
:101210005AD0181CC7300178C9B2002908D0037809
:101220005BB2022B00D0012313700023037070E126
:101230001D1CC4352C78002C09D0012414701A1CF4
:10124000C532D033017029701170196062E10498C1
:10125000002839D1191CD0310C68002C09DD013C63
:10126000012C01D00C602FE0049B0B600323137052
:1012700050E11A1CFC3212681188764A914223D040
:101280001A1CDC321188744A126852888A421BD8B0
:101290006F4C2068427C181CCC300068904213DBF5
:1012A00007AA1180DE331B886C49538002234B70E0
:1012B000CB70049815230B7106F016F8634B226867
:1012C0001B68927CD0331A60614C2768F87C002838
:1012D00000D01EE104995D4D002900D082E02C6809
:1012E000231CFB331B78002B56D03B1C2C331B7864
:1012F000002B51D0231C0791F0331B680393231C50
:10130000DC3303981A8843009A533B1C2D33197819
:1013100004984B00F618031C994206D05A00B21AE2
:10132000023A128801338018F6E7FEF711FF0790A2
:10133000FA8B231CF433904202DA1A68013200E07F
:1013400000221A603A1C2E3212781B68934215DD77
:1013500042497C235B42CB7007AA1623012400205C
:101360000B714C7005F0C0FF2B6800201A1CF03286
:10137000F4331060186005F0F9FFCBE03B1C2D330F
:101380001A780399231C013AF033914202DA0A1CBD
:10139000013200E000221A60D8340137FB7F226856
:1013A0009A4217DB2E4900201223021C0B7105F014
:1013B0009BFF2A682648131CD43319680068013142
:1013C00019600230C07F814204DB00211960C832FD
:1013D000022313702A680023111CC631D8320B7007
:1013E000136047E02B681A1CD03210602A32127842
:1013F000002A3FD0191CDC31098807AA1180DE338E
:101400001B881649538002234B70CB7019230B7134
:1014100005F06AFF2B682268191CDC310C88D08B20
:10142000163984421ED2181CDE300488508D844246
:1014300018D2097800291DD1D83301321968D27F1A
:10144000914217DA0131196014E0C0460000002013
:101450000C0F0020FFFF0000100F00201C010020D7
:101460004F04002001220A70191C0022D831D43305
:101470000A601A60294D2B681A1CFA321278002A69
:1014800047D105980279002A41D01A1CC432147839
:10149000002C3ED1224E186B3768798BBA8BFB8AB1
:1014A0003F8B009705F0ECFF36682B68718CB28C8F
:1014B000071C186BF38C368D009605F0E1FF2B6846
:1014C0001A1CDC321188DE33B94202DA1A888242F1
:1014D00010DB07AA11801B881249538002234B702E
:1014E000CB70002017230B7105F0FEFE2B68012244
:1014F000C5331A702B681A1CC5321278002A08D01E
:101500000499002905D0C43301221A7002E0C533C2
:101510001A700124201C09B0F0BDC0460000002054
:101520000C0F00201C010020F0B591B002AF03F0B9
:10153000D7F9061C03F0ECF9386103F0DDF9B14B83
:10154000B8601C686846E36800211A1C0E32D20895
:10155000D200801A226985460E32D208D200801A43
:1015600002AD8546FD6102AD7D6272799A18131C49
:101570000E33DB08DB00C01A53000E33DB08DB0040
:101580008546C01A02AD8546C01ABD6102AD8546CA
:1015900002A87861B86908F0BDFAE1687279281C80
:1015A000521801215200494208F0B4FAE3687279F6
:1015B0009549D2185200786908F0ACFAE2683969A6
:1015C000F8693D6308F064FA3D69F020800029184D
:1015D0002269786A4024002508F05AFAFC603D62CE
:1015E000796AF86904F02EFE032003F0A3FF854D0D
:1015F00086492B68864C5A6818684A709A68042392
:10160000CB7051230B7123688A705B6901329200A1
:1016100008709A18022005F067FE2B687D491B6947
:1016200004254B705A230B71236802201A6ACD706F
:1016300005F05AFEB479013C631C2CD07579013D4C
:101640006A1CF8D0737978696343EB185B001A5A07
:10165000714B9A42F3D0B96930227960F9627863AC
:10166000D219694609CA09C1211C7B68F8692A1C7C
:10167000FEF776FF002803D03B6A01339BB23B6242
:101680007379BA6963433869EB18D15CC25C8A1814
:10169000F969CA54D3E7F479013C601C30D0B179C0
:1016A00073797D694B43E3185B005A5B5A4B9A424E
:1016B000F2D0BD6930207D60FD62C0197D6984462D
:1016C0007D636846624628CA28C0221C7B68786A07
:1016D000FEF746FF002803D03B6A01339BB23B6212
:1016E0007379B279BD695A432B193D69F0202919E4
:1016F000800009189A5C0B787D6AD3182B55CBE7CC
:10170000404B3C6A1B68DA681B69D3189C4206DAB6
:10171000FB68013BDBB2FB60002B00D060E73B4C79
:10172000B3797F252370737980206370A370E37889
:101730004042AB4301252B430343E3700820D223EF
:10174000211CFA69237105F0CFFD3249F3797F221C
:101750004B70CB78082093431D4380235B421D438D
:101760007A6AD323CD700B7105F0BEFDB379251CC9
:10177000013B0FD37279013AFAD37179FC6959436D
:1017800089186118BC68E018A4300C78007820181B
:101790000870F0E7F379013B08D3BC68E2187C6A73
:1017A000C8321178E25C8A18E254F4E7F869796A81
:1017B00004F048FDB3797F202B70737901216B70A1
:1017C000AB70EB78802483430B4364422343EB707C
:1017D000291C1D23FA6908202B7105F085FD0D4990
:1017E000F3797F224B70CB78012593431D432C4323
:1017F0001E2308207A6ACC700B7105F075FDBD467A
:101800000FB0F0BD0C030020FFFF000048040020D3
:10181000000000201C010020FEFF000008B503F0BE
:101820006BF898300378002B02D1FFF77DFE01E0C2
:1018300004F0AEF808BD0000F0B593B002AF05F0BB
:1018400029FC2621C85508F091F808F0C1F801F0EC
:10185000EBFBFEF7CDFF05F01DFC2722041CD05545
:10186000052800D100E116D8022800D1BCE007D835
:10187000002828D0012800D010E205F067FCA6E07F
:10188000032800D1DEE0042800D007E205F05EFC6A
:1018900001F002FAE1E0092800D108E108D80728A0
:1018A00000D1ECE0082800D0F8E105F04FFCF2E0B0
:1018B0000B2800D1E1E100D20DE10C2800D0EDE1D0
:1018C00005F044FCE4E105F003FC051E31D00128DD
:1018D00000D0E3E1BC4DBD482B68196A1B69F96172
:1018E000BB6102F0F7FF06F063F9061C05F004FE89
:1018F000786108F017F8331CB54AD8331A807A6932
:10190000B44B736014702B6803CB03F0E3F804F05E
:101910003BFDB148343002F0F5FF2B680A22AF4995
:101920001A621C61201C3F23221C0B7105F0DCFC99
:1019300037E008F01BF808F04BF8FEF759FF281CB9
:1019400007F0DAFF02F0DEFF0124012C02D0022CA6
:101950000AD014E0002000F0ABF903F0D5FBC0B2D0
:1019600005F010FDFFF75AFF9D4B381C391C009302
:101970002730263100229B4B00F04EFE041C05F060
:10198000A7FB002800D089E105F084FB2725EB5D4B
:101990008342DAD082E105F07DFB2721CB5D8342D3
:1019A0000FD1FFF73BFF8E4B381C391C00932631BB
:1019B00001228C4B273000F02BFF05F089FB01281A
:1019C000E9D02B68FC69BD691C621D6166E105F008
:1019D00061FB2722D35D8342F9D007F0A3FFFEF716
:1019E00007FF05F04BFA59E1FFF736FB05F018FB4E
:1019F000002003F025FE03F0B7FDFEF77FFDFFF7A3
:101A00000DFF05F0A3FB05F0ABFB04280CD004D8B8
:101A100000280ED001F042F90BE0052807D0062877
:101A200007D103F051F904E005F064F801E003F098
:101A300039F905F02FFB2724E35D8342E3D0FFF75C
:101A40001AFB2BE105F082FBFFF7E8FE05F022FB15
:101A50002725EB5D8342F9D020E105F01BFB272110
:101A6000CB5D8342F9D019E105F070FB03F0D4FEA1
:101A700005F010FB2722D35D8342F9D00EE105F07B
:101A800065FB012000F014F905F004FB2724E35D59
:101A90008342F9D002E1002003F04CFD03F0DEFDAB
:101AA00005F0F8FA2725EB5D8342F4D0F6E005F067
:101AB0004DFB002003F000F8002003F03BFD03F095
:101AC000CDFD05F0E7FA2721CB5D8342F4D001205C
:101AD00002F0F2FFE2E06C4600207C6107F0AEFF0E
:101AE00007F076FF002003F0ABFD374D2B68196837
:101AF0005E681B694E43F3180733DB08DB00E21A0C
:101B0000954602ACA6193C6002F0EAFE02F000FF26
:101B100002F0F2FE3868311CBE6103F007FF2B684B
:101B20006D465A681B69D3189B000A33DB08DB003B
:101B3000ED1AAD4602ACFC6105F008FB224D2821F0
:101B40002B6829241A680420CA551A792A21E255DB
:101B5000CA555A1DD27F1B692B242C21E255CB5527
:101B60002D2201233C68D355391C0022131C283137
:101B7000009405F07FFB3868B96904F063FB00202E
:101B800003F0D8FC2B6818485D680668BD60002229
:101B9000BD68AA4206DAF56991006D58FC69013208
:101BA0006550F5E7FC69AA001969A4180668796010
:101BB000A44600227C68A24218DA756A90002D586B
:101BC00061460D500132F5E70C030020509B0000E8
:101BD00076020000A1030000D09B00004F0400200B
:101BE00034030020180F002000000020BC68196892
:101BF0003122D45530259A68E9553225EA55053306
:101C0000DB7F7C683321CB553423DC55264B0132F6
:101C10001B6892005B6904259A183521CD55009206
:101C2000391C0022131C0220303105F023FB012354
:101C30003822D3551D4B39241B683A211A791020BC
:101C4000E255CA555A1DD27F1B693B24E2553C21FF
:101C50003D22FC69CB55D555391C0022131C383167
:101C6000009405F007FB05F015FA2725EB5D83428C
:101C700000D163E77C69A54610E005F067FAFEF73E
:101C8000F7FC05F007FA2725EB5D8342F7D005E066
:101C900005F000FA2721CB5D8342F9D02722D35DDE
:101CA0002624E355D7E5C046000000200C030020A1
:101CB000F0B5D14C9BB0236800AF9B6878617B6224
:101CC0005B0001333B6503F00FFA2368FF229B683A
:101CD000F865D31A984200DDFB65F86D7C6A041B39
:101CE0003C626C4603F008FAFC643C6D6846650093
:101CF0002B1C0833DB08C14CDB00C01A01236370C6
:101D00007C235B423A1C8546E370211CB1230020F2
:101D10005C3223716E4605F0E7FA0023211C3C6D0E
:101D2000A34205DA3C6A5A001819B0520133F6E7AB
:101D3000E4B24C70FC610024321C0223201CCB70E6
:101D40000C7105F0D1FA2B1CF86C08338546DB08C2
:101D5000DB006946C91A8D46C91A68468D46B963C3
:101D6000386403F0A3FD3861012003F05BF8211C07
:101D70002A1CB86B07F0CEFE211C2A1C386C07F019
:101D8000C9FE3B6D68469B00BB610A33DB08DB0084
:101D9000C01A396985466A46C01A89007A63854641
:101DA0003863B960FC640021BA69786B07F0B2FE51
:101DB000386BFF21BA6907F0ADFE00248E4B7C65BD
:101DC0001B687C6D5B689C424ADA3C6A0026E4B280
:101DD000201CFC6303F09DF903F066F903F018F88A
:101DE0003C6B7D6B386D0136F217C30F8642534151
:101DF000DBB2FB62002B06D1F96B8819C0B203F08D
:101E000088F903F051F96B46FB60BB686A460A33F8
:101E1000DB08DB00D01A85466A46BA6403F04EFD43
:101E200000231A1C39698A4205DAB86C91004158BE
:101E300001325B18F6E72A68934200D92B602068CC
:101E4000834200D22360F968FA6A8D46043404356F
:101E5000002A02D102F0DCFFC4E77C6D0134ADE75B
:101E60000024674D7C653B6D9C4217DA796B3A6BB9
:101E7000A300C858D358C01A854204DD3B6A051C2C
:101E8000E318BB627C64796D814200DA786502F008
:101E9000B3FF3A6C6300D0520134E4E7786D02F08E
:101EA000ABFF554B1B685B88984206DA7C69012CB6
:101EB00003D0FC6DBC627C6A7C64524D32222C687B
:101EC000796C231C8C335A6064229A6001220220B0
:101ED0005A613A6B81408A58002618611E60101CB6
:101EE000DE607A60F96302F087FFA434FB6B796BE4
:101EF000206058582C6802F07FFF2B68AC342060BB
:101F00001A1C41497C69B832C03311601E60012C33
:101F100022D1BA6B331C3C6DA34209DA3C6C5900E8
:101F2000615A1088884200D2118001330232F2E7F0
:101F30007C6C6300BC6B1A5BFC6C131CA24200D26D
:101F4000231C2E499BB2FC69FB64002002234C70C9
:101F5000CB700871BA6B0CE0786D02F04DFF274929
:101F600080B2FC69F8643A6C0220C8704C700E7143
:101F7000301C05F0B9F97C6C6021CC53BC6A62203E
:101F8000C453786C396C44000C192388F86C6422B3
:101F90001A49D3536623D85304234B703A1C0223A7
:101FA000CB706032B22300200B7105F09DF92388BD
:101FB000144C2268111CFC3109680988994227D207
:101FC00007F042FD051C07F0A1FC0378061C002B5E
:101FD00007D0012005F0CAF923680236FC331E60E1
:101FE00027E0002D25D1094B1B68DB7C002B20D17D
:101FF000012005F0AFF91CE0100F00201C010020AB
:10200000FFFFFF7F00000020FFFF00000C0F0020FB
:10201000FB321278002A0CD00E4D29684A889A4269
:1020200007D9002005F0A2F923682A68FC330232A0
:102030001A607C69002C06D1BC6AE0B203F069F832
:10204000BD461BB0F0BD05F025F8072800D1AAE673
:10205000F2E7C046100F0020F0B585B00092039162
:10206000029007F0F1FC061C05F050F8071C05F083
:1020700055F8734D01902B681A1CF8321278BA4249
:1020800020D0002F08D06F4900203B23021C0B7189
:10209000022605F029F910E001993C1C00290DD118
:1020A00068493C23381C3A1C0B7105F01DF92B685C
:1020B000FA331E78731E9E41F6B201242B68F83362
:1020C0001F701DE01A1CF932127801998A4216D04D
:1020D000002906D1FA331E78731E9E41F6B23A23C8
:1020E00001E03923022657490020021C0B7105F03C
:1020F000FBF82B68019AF9331A70012400E00024E0
:1021000004F0D8FF071C04F0F9FF009B032B02D05A
:10211000002F03D107E00124002F36D0002004F067
:10212000D1FF012431E02B68F8331F88002F2CD118
:102130000099012902D0022904D00EE0009805F090
:1021400009F90AE0381C05F005F92B68FB331B7808
:10215000002B02D0381C05F009F905F0F5F82B68C2
:10216000071CFA331B7883420FD0002802D01123BA
:10217000012601E01223061C32490020021C0B71CB
:1021800005F0B2F82B68FA331F7007F05DFCB0421F
:1021900039D007F059FC07F0A3FB071C301C07F0EF
:1021A0009FFB009007F050FC301C07F047FC07F045
:1021B0000FFC254B1B681B7D002B10D0012C0ED073
:1021C000009B3A1C9B329B330399029805F0CCFA92
:1021D000002003F0AFF90024FEF722FB06E02B6895
:1021E0000020E033187003F02BFA0124002005F0E2
:1021F000BDF82B6800211A1CFB321170134AFC3306
:10220000126802321A6007F01FFC07F07FFB0378A8
:10221000002B08D005F0A4F82B68FB331A78824213
:1022200001D01870012404F081FF051C05F0DCFCCE
:102230000379AB4200D00571201C05B0F0BDC0464B
:10224000000000204F0400200C0F0020100F002081
:10225000F7B5434C151C236801911A1CC53212783E
:10226000061C002A23D01A1CFA321278002A1ED12A
:102270001A1CE0321178002919D1C4331B78002BC5
:1022800015D10123137002F037FB071C02F028FB65
:102290003A1C031C9B325D33301C019905F064FA33
:1022A00003F014F9022003F01DF9FEF7B9FA2368D0
:1022B0001A1CE0321278002A4FD01A1C294F002035
:1022C000C43210703A680190126A011C013A0ED3B0
:1022D0000E265643B446AC446646B688002EF5D06A
:1022E00036B20131B042F1DA301C0192EEE71A1C2D
:1022F000FA321278002A13D1012911DD05F074FC9D
:102300000123B03003603B681B6A013B0AD3019E86
:10231000B342FAD00E225A430021AA189180F4E762
:10232000002904D023680022E8331A6008E01A1C50
:10233000E832E43311681B68994201DC0131116015
:102340002368191C1A1CE831E432096812689142AA
:1023500005DDC43301221A7001E0E8331A60F7BDCD
:10236000000000200C030020F0B5A34C93B002AF96
:102370007A6222687B60136892689D1C5200554304
:10238000F9606946B9605208291C0133534308318A
:10239000C9089A4E3861C9006846401A854601331B
:1023A000306802A95B00CB18F9613C220021303073
:1023B0007B6107F0AFFB2A1C0021F86907F0AAFB3C
:1023C0008F490020A623021C0B7104F08DFFFEF73D
:1023D0007DFE3168081CDC30DE31FEF749FA2368E7
:1023E000884D5B6804226B705B232B713368EA7045
:1023F000291CDA69022004F077FF2368291C1B6975
:1024000002206B700423EB706C232B713368002562
:102410005A6A04F069FF33687B491A1CDC3212885F
:10242000DE337A631B883A1CBB630C2001233432F1
:102430000B71FD6304F058FF23682C2019682D22CE
:10244000C15558682E21D0559A682F20CA55591D5C
:10245000C97F1B69C1553021CB5504203123D85584
:10246000336801325B6992009A18391C009202208D
:102470002C312A1C2B1C04F0FDFE396E0D700091CE
:10248000FA6D01923869F968FA697B69FEF7CAFB4F
:10249000F861A84200D08CE026686846F16AB8610D
:1024A0000A01131C0833C01A854602ADF969281CBD
:1024B00007F030FBF26A281C796AFEF75FFD23689B
:1024C00069469A6A0E235A43131C0833DB08DB0063
:1024D000C91A8D4602ACF969201C07F01BFB7B680A
:1024E000281C211C7A6AFEF785FDB86DFEF760FE98
:1024F000464B1B681B7D002B04D13869F968221CF0
:10250000FFF7A6FE201C796A01F05CF8201C796AAE
:1025100000F0AEFE06F056FE83000733DB08DB005A
:102520006A46D21A954602AB7B61334B061C1D6886
:102530000E22A86A3E62031C013B5343E4187862F2
:102540000434786A013878620FD30021635E002B6F
:1025500009DD3A6A7B69013A90003A621818211D38
:10256000042207F095FA0E3CEBE72A683421CA559D
:1025700068683523D855AB683621CB550535EA7FD9
:102580003720C25538210022CA551C490133096839
:102590007E22C96A5B00CB1852423920C255391CD1
:1025A00000933431F2B203207B6904F063FEB96911
:1025B0008D46BA68954602F025FE02F087FF02F0CC
:1025C000F9FB012002F0B6FF02F040FD0B4BC822E0
:1025D0001B6838699A56F968FFF73EFD002800D15C
:1025E000F8690B4B1A680B4B9A4202D003F014F9AE
:1025F000FEE7BD4611B0F0BD0C0300200000002036
:102600004F0400201C010020230100200C0F00209B
:1026100068100020CDCDCDCDF0B55B4C8DB004AFB2
:10262000FB60236879601E6859683A604E430A224D
:102630009A622822DA621B696A46F3189B000A3301
:10264000DB08DB00D21A954604AB3861BB6105F0AC
:10265000D1FA236869469C6AB600E200131C08336D
:10266000C91A8D4604ABA400FB61231C0833DB08A8
:10267000DB00C91A8D4604A9B960F869002107F08A
:1026800049FA221C0021B86807F044FA3F4D0024A3
:102690002B686946FF335C713D4B1B682D331A78FC
:1026A0005200131C0833DB08DB00C91A8D4604AB4B
:1026B000181C211C7B6107F02DFA04F01DFFB9697D
:1026C000BA698E19331C4178201CFEF78BF9012062
:1026D00003F042FB2B68F9689A69201CFEF7CEF9DB
:1026E000201C03F039FB7B6839691A780B789A4211
:1026F00005D004F02BFD3A69796813780B702B68CC
:1027000000229A6004F038FE041C02F0FDFCA04296
:1027100004D0201C02F0FDFC022422E07A69009221
:10272000FB680193B96B0291FA69311CBB68B86907
:10273000FFF71AFE154B174A1B68041C9968914253
:1027400002D09A6801329A6000280AD104F0C0FCD5
:102750003A68904205D104F09DFC39690B788342B8
:10276000D0D0F869FEF79DFC02F0BAF8051C02F023
:10277000C3F82A1C011C9B31F868AC3205F030F814
:10278000201CBD4609B0F0BD0C0300200000002055
:102790000C0F0020FFFFFF7FF0B51B4B87B01B68BD
:1027A00002AF396019689B680E1C5B0002365E43FD
:1027B000151C321C5B080832BB60D208134BF96051
:1027C000D20069467860891A18688D4602AC0021EB
:1027D0003C22303007F09EF9321C201C002107F00B
:1027E00099F900232B70FB68BA6801335343013316
:1027F00000955B00E31878683968221CFEF712FA2E
:10280000BD46C0B205B0F0BD0C03002000000020A2
:10281000F0B5D44C0E1CA54402AFF860D2483A6023
:102820003B6203F00BF902F06DFA02F08DFA02F050
:10283000E9FCCE4B0A221B68052459681D689A6280
:102840004D43DC621B69EB189B009B18DB08DB0027
:102850006A46D21A954602ABFB6102F05FF8031C90
:10286000B8331B687861BB6005F0C4F9381C0021DF
:102870005022783007F04EF9381C002128225030C1
:1028800007F048F93B1CC833BB6404F035FE78639D
:1028900003F08CFAF969AD004D193D617D6B3B6920
:1028A0006978201CFA69FEF79DF803F0A3FF8821E0
:1028B0008900C9590B78002B06D1AD4B04201B6849
:1028C000396A5A69FEF7DAF8FD6832782B789A424D
:1028D00003D004F03BFC2B783370A6490020A223E0
:1028E000021C0B7104F000FDA14B1A6800239360D9
:1028F0001E1C7B627B63FB6204F03EFD386302F0CA
:1029000003FC3D6BA84205D0281C022502F001FC07
:102910003D63ABE1002E00D094E0944B6D461B6804
:102920007D609A6951005A6901324A43131C083389
:10293000DB08DB00ED1AAD4602AD281C311CBD6280
:1029400007F0E8F8796B8A4D082910D103F052FF9F
:1029500088229200D2597E631378002B6DD12B68A8
:1029600004205A69396AFEF789F87E6365E003F04E
:1029700041FF3C1C042002F0DDFD3C342B68267036
:1029800088255969AD000094B86A3A6AEB5904F099
:10299000B3FFB861012812D1E91909680D78002D3B
:1029A0000DD103F003FA052002F0C4FD7149A32301
:1029B000301C321C0B7104F097FCBE693CE023789C
:1029C000002B38D188229200D2591378002B04D1E1
:1029D000386AB96A642205F081F8674B7D6A1B6822
:1029E00033331B785B009D420BDD03F0DFF90025DC
:1029F00005200121FA693B69FDF7F4FF03F0FAFEB7
:102A00007D627D6A01357D6202F0E6FD02F098FB91
:102A1000594B1B683333187802F080F9002002F01C
:102A20009FF9386B02F075FB02F0AEFB7B69BD6865
:102A3000B8331D6001E008257D637D68AD46002543
:102A40003D63B5E04C4B01261B6834331878484B86
:102A50001B68186002F062F9052002F043FD88232C
:102A60009B00F8693969DA59FFF796FE3863002848
:102A700000D09DE03D4D69462E68B962F36A1A01A7
:102A8000131C0833C91A8D4602AC201C396B07F0A1
:102A900041F8391CF26A201C7831FEF76FFA2B6876
:102AA0006D469A6A0E235A43131C0833DB08DB0079
:102AB000ED1AAD4602AD396B281C07F02BF83A1C15
:102AC0003B1C201C291C78325033FEF793FA2E1C35
:102AD0000A24B11C301C013C06F0C8FA0E36002C4A
:102AE000F7D1391C281C7A6B483106F093FB031C84
:102AF000013BFD6ADBB201229A429B411D40786393
:102B0000FD62032803D0072811D1182405E0381CE2
:102B1000483006F077FE041E0FD004F0E1FA164BA1
:102B20001B689B6B18400123A340034205D0FD6A3C
:102B3000B42D56DC002C03D00BE0FD6AB42D50DC24
:102B400002F0C4FC02F05EFBFD6A01260135FD6265
:102B50002CE00221172C11D13C223D23D155DC550C
:102B6000D01910E0ECFDFFFF400D03000C03002026
:102B7000000000204F0400200C0F00203C253D22C7
:102B8000E955D455E81904F04DFB02F09FFC0120F3
:102B900002F0B8F83C490020A223021C08250B7162
:102BA000002604F0A1FB03F025FE7D63BD6AAD465F
:102BB000364B374A1B689968914202D09A680132B5
:102BC0009A603D6B002D51D104F082FA3D68A84215
:102BD0004CD104F05FFAFD682B78834200D18BE67C
:102BE00044E004F0ABFA00282DD00224381C221C4B
:102BF00028493C3006F04CFF381C211C3C3004F0C6
:102C000011FB052004F030FB4C21CB5D4022D35555
:102C100042254123EC55DC55442200234525432120
:102C2000D355EA5DCB557F218A431443802252421B
:102C300014433A1CE919C8320C700520009205397A
:102C40001A1C04F017FB02F041FC012002F05AF8B4
:102C50000D490020A223021C002608250B7104F058
:102C600043FB03F0C7FD7D63FE629FE77B69BD68A0
:102C7000B8331D6002F02AFC03F098F8386BBD46AB
:102C800083239B009D44F0BD4F04002000000020E2
:102C9000FFFFFF7FCC9F000070470000F0B5CC4DD8
:102CA00099B02B6800AF5C68F8641868BC63604337
:102CB000021951000831C9086600C9006C46641A3F
:102CC00091000A31BE647863A546FC624600C908DB
:102CD000201CBC6BC9000732401AA400D2083C6318
:102CE000D200441A85467864A01AA5468546DA685B
:102CF000BC6200216C463C6206F00CFF2B68786BCE
:102D00001A690021684406F005FF2B680021DA6883
:102D1000786C920006F0FEFE2B68786B1A69796C6D
:102D2000840092000819002106F0F4FE2B68A949DE
:102D3000DA68B86A920006F0EDFE2B68BA6AA54917
:102D400010191A69920006F0E5FEFDF7BFFBFD6C55
:102D5000022D05D0032D05D02F30012D05D102E025
:102D6000303000E031300078F8633D6BAD08FD6134
:102D7000BD6C6D08BD61FD6B013D3D637D6C2D1922
:102D80007D6275083D61FD6AAE19FE60BE6A341948
:102D90007C613D6B8E4C013500D1AAE0002002F031
:102DA000C9FB25688C4B6C681E68013C5DD3A00094
:102DB0002B68B860591EB964F7D3A96872694B4390
:102DC000E31801339B009858FB6C022B0AD0032BAD
:102DD00022D0012B47D1F169BA688B58C01AC3437E
:102DE000DB171840B96CFB697A6C4B43E3189B0006
:102DF0009A58796C80183A6B5850002A33D1B96CC4
:102E0000BB694B43E3185B00F96B3B64FDF752F978
:102E10003A6CFB6AD05226E0B96CFA694A43A318AF
:102E200099007B6CC958031E8B4200D20B1C796C35
:102E3000A21892005350B96A5258904200D9101CFF
:102E4000B96CFA694A43B96AA21892005050181A2C
:102E50007F22FD2801D84008C2B23B6AB86C19191C
:102E6000BB6B4343CA54BB6CA4E72E695A4B741E18
:102E70001D68A400013E38D32A6AFB6C1059022B4E
:102E800009D0032B16D0012B2DD1696A0B59C01A1A
:102E9000C343DB1718407A6A7B6A1259396B801872
:102EA000185100291FD1F96BFDF704F9FA68730076
:102EB000D05218E07B6A1A59031E934200D2131CA9
:102EC000796A0B5179690A59904200D9101C7A69C4
:102ED0001051181A7F22FD2801D84008C2B2386A62
:102EE000796B43189A55043CC4E73C6B013C3C6346
:102EF0004FE7FE6AFD6CBE64022D06D0032D61D043
:102F0000012D6DD100F00EF96AE001F0E9FC381CEA
:102F100032491022503006F0BBFD02F065FD2168F9
:102F20002D4B0E68F863BD691868331C013B5D4387
:102F3000FE6484467D64FE6C013EFE6422D34B68D1
:102F40007E6CFD6AF01840005E002818BE63002207
:102F5000023A013B11D3FD6BBE6B6D003D646546CB
:102F6000ED69B6187E63760076593D6C5035ED5BA1
:102F7000AE1B855A75198552EAE77E6CBD69761BD2
:102F80007E64D8E70B693E69134AF118FE6A49006E
:102F9000580015687118F8640022023A013B0ED3FC
:102FA000FE6CB0186E6A400080598E5A361AB446CC
:102FB000FE6B70005030C05B60448852EDE700F05B
:102FC000B2F80DE03D6ABD6400F0AEF8012308E000
:102FD0000C030020FFFF000000000020CE9F000037
:102FE00002232268502610685124F0551179522589
:102FF000E155E955511DC97F5326F15512695420F9
:103000005521C255CA5D7F218A4313438022524213
:10301000381C134350305522B96CD35504F0A8F82E
:10302000BD4619B0F0BDC04608B503F091FF08BD1C
:1030300038B504F0D9FD234B1B681A6B002A03DD59
:10304000996BCA420AD510E0002A07D11E490968C7
:1030500014254C5F9D6B0121A54207DB1B4904240D
:1030600009788C428941494200E001211C1C7834D6
:103070002170052A12DDD96B13291FDCD2225200E0
:1030800081580A1C013A1CD3940004197D34FF3482
:103090002468012CF6DC0129F4DD0CE0032A0DDCA8
:1030A000DA6B0C2A0ADCD22252008258002A05DD93
:1030B0005D6C022D05DC7933012201E079330022B9
:1030C0001A7038BD00000020100F0020140F0020DF
:1030D00010B504F06DFD124B1B68196B1A1CFF3202
:1030E000002915DD041CF0342488A14210DA642480
:1030F000EE30614300889C6B6043C14208D5191CC7
:10310000FA310978002901D1012100E00021517133
:103110005279002A02D0783300221A7010BDC046BE
:1031200000000020704770477047000008B502F0AB
:103130001BFA01F0FDFC01F0ADFC01F061FC0F4B4E
:103140001B681A7A0E4B1B68FC33002A01D002223E
:1031500000E003220B491A6100230B700A49A022E8
:103160000B700A49D2050B709363D36B9B0E9B06C1
:10317000D36362B603F008F908BDC04640100020D2
:103180001401002029000050280000502A0000509F
:1031900038B5041CFDF7ACF9051C04F009FD291C29
:1031A000FF314B79002B24D0124B00221B68DB6AC5
:1031B000013B07D3180120180825405F0028F7D1EC
:1031C0000122F5E70C4B1B68186B002811D19D6B91
:1031D000002D0ED1FC33002A0AD0DA68FE2A01DC69
:1031E0000132DA60DB68052B03DD00234B7100E060
:1031F000DA6038BD0C0300200000002070B5051C0B
:103200000C1C161C03F0D6FF002802D001280AD09F
:103210002DE00E225643AD19EA88FF23FE2A00D87E
:10322000D3B2637123E00E227243AA18D188FF2320
:10323000FE2900D8CBB263710B250A23D35655570C
:103240000926ED1A08239657D356F61AB54207DD1C
:10325000281C0521FCF77CFF4519A571E67106E0E5
:10326000301C0521FCF774FF8619A671E57170BD4D
:10327000F0B5C34B8DB01B6806909F68079105970A
:10328000DF6803971F6904975F6902979F6903F0DE
:1032900097FFBC4B01201B68F8331B780190002B73
:1032A00059D00021079D069C01910E1CB64B1B684E
:1032B0001B6A9E424FDA2B8809A803806B884380E3
:1032C00005F002FF0422A35E002B40DD2388684640
:1032D00003846388438408A805F0F6FE6A46202329
:1032E000D35E059898420BDA0399994208DD684647
:1032F0002222825E0499914202DA0298904221DCF5
:1033000004216A5E002A1ADDA04A1268921940322E
:10331000127852B2012A12DD0598C21B9A420EDAC7
:103320000399CA199A420ADD6A462223D35E049899
:10333000C21B9A4203DA0299CA199A4205DC002399
:10334000A38004E00122019201E0012301930136F0
:1033500008350E34AAE70127069D079C0297002630
:10336000894B1B68186A864200DBD1E0238809AFCD
:103370003B806388381C7B8005F0A6FE04202B5E12
:10338000002B00DC95E02B8869460B846B8808A82D
:103390004B8405F099FE6B461B8C6A460393528C56
:1033A0000020395E10B2049205900222B85E059F9B
:1033B0001BB2381AC217591A80185040CA178F18F2
:1033C0005740724A00971768BA19783212799446B2
:1033D0006F4A61461268002901D14C3200E04D323B
:1033E0003F79127807970421675EA9888C46079970
:1033F000002913D1002F05DD904203DA009F974288
:1034000000DA7AE0019F002F77D00E2B75DD5C4A41
:10341000126812680E3A9A426FDD09E0002F04DD4F
:10342000904202DA009F974267DB019F002F64D031
:103430000AAF3A78802040421043DF210840297BC0
:1034400001221140402210431022904309010F2213
:1034500001430298914301431B12397013400793B3
:10346000059B79781812079B91430B431340000189
:103470001843787003986346B87004991AB2F970CB
:10348000FF2A00DDFF233B71321C0698391CFFF731
:10349000B5FE381C03F09EFE0423E25E3B4B1B6826
:1034A0009B197833002A01DD012200E000221A7105
:1034B0001DE00420235E002B1FDD0AA800230299D3
:1034C000436040230B4303703A880123FB56039269
:1034D000032179569C4662467B880F2717400901D5
:1034E0003943039F41708770C37003F073FE2B88CC
:1034F00023806B886380EB88E380AB88029AA3808B
:1035000001320F231A4001360E350834029227E7A4
:103510001B690F255C1E1D401C4E621C3AD0316891
:103520006700CB191A1C90320020125E8633002AE5
:103530000FDC1B881AB2002A16DD00210AA80A91A6
:103540004160802129430170FF2A00DDFF230371C0
:1035500008E000215B5E002B06DC0AA800230A932A
:103560004360057003F036FE3368013CDF193B1CF5
:1035700086373A8890331A80013D0F23CBE7C04647
:103580005C100020000000200C0300201403002029
:1035900058100020336801201A1CB032116808321C
:1035A000002902D11068441EA0411C1CA6342070C2
:1035B0001268181CB430BC3301601A6003F01EFEA0
:1035C0000DB0F0BD70B5124B051C1B680C1CF2331E
:1035D0001B78002B1BD00F4A1368161C191CB43122
:1035E0000968002905DDBC331B68002B01D105F0FB
:1035F000ABFA33681A1CBC321268002A07DDB433F8
:103600001B68002B03D1281C211C05F073FA70BD28
:103610005C10002014030020F0B591B00E910890CA
:1036200003F076FF04F0DAFACC4B01211B68089C0A
:103630001A1C5A321278002591401A1C5B321278FB
:103640005C33891A1A780A958B1ADBB20F93C44B34
:103650000E221B680B950C93C0330D93C14B196858
:103660000B6A5A43A2180E3A013B0BD3D4880A9E28
:10367000A64200DA0A940427D45F0B9DA542F2DA31
:103680000B94F0E7B84B3E301B68FF335B7B012B9C
:1036900001D1042300E0022303700B6A089F013B61
:1036A0000593059E0E237343FB1806330793059F6E
:1036B000013700D1C7E0079C023C0025635F0694F8
:1036C000002B00D1B8E0A54C23684E331D7803F0E1
:1036D000FFFC079E031C3088002B08D123681A1CAE
:1036E00019691432243303F0DCFE041C07E023685C
:1036F0001A1C19691432243303F0D3FE4400FCF77A
:10370000F7FEFF304279954B002A05D01A68353212
:103710001278944200DA141C1B681A1C4F3212787B
:10372000002A01D1642245E02A1C0C9D7535FF3525
:10373000287800281CD1069F64210026BE5F171C34
:10374000714367438C460C996D31FF31BC450DDDEB
:10375000A6420BDC854F0E683F6801360E60DA37F3
:103760003F78BE4204D101262E7000E000200860A0
:103770000C987530FF300178002915D0069E0C9901
:103780000025755F6D31FF31A5420BDD0D681E1CF4
:1037900001350D603E363678B54205D100250570FD
:1037A0000D6001E0002008600C997531FF31097847
:1037B0000029B7D06A49059F0968069DC81940309D
:1037C00006780020285E002E05D01D1C3E352D7881
:1037D00076B2AE421ADC642545435443A5420FDB62
:1037E0001A1C443212780A9F079E7A433488921139
:1037F000944205DB9B6C0B9C63439B1198421BDA44
:10380000079D069E00232B8033800CE034331B7809
:10381000574D5C436843624390420DDA079F069C14
:1038200000233B802380059A143292008A18B0311D
:1038300053600B68013B0B60059D079E013D0E3EEA
:103840000595079633E7464B00221B680E9DB03363
:103850001A60444B1B681B6A5C1E0594059EE200BF
:103860000E247443AF18089D0C2272432C193F3369
:103870000C9D0D9E5B00EB18B218C23307920A93A1
:10388000059E374D013600D102E20426A35F334A7C
:10389000002B00D1BDE1059E2D681268A9190B1CF3
:1038A000403318783E320130C0B21870127840B2FE
:1038B000961DB04201DD04321A704023CB56012B15
:1038C00005D123883B8063887B80E388FB80059E4D
:1038D000AB1940269E57012E00DC82E1B01C03216B
:1038E000FCF78CFC0B91022E44D11E4B00203A5E5B
:1038F0001E6802217B5E69692D6930686D10551B59
:1039000076688C46E917013E6D1836024D40761BED
:103910007F2E0ADD65466910591ACE1701388919BC
:1039200000027140401A7F280DDC0021605E801A81
:103930000222A15EC91A04F0B1FD0B2803D93B880D
:1039400023807B8863800323013B1BD32188079D51
:103950005A00A9526188AA18D180F5E758100020B2
:10396000140300200C030020000000205C10002045
:10397000102700000B9E079D3A887300EB181A80F1
:103980007A88DA80D34B059E1B680221655E9B19FD
:1039900040331B780020265E5BB20893032B00DCCB
:1039A00015E10B9A07985300C3181988101C0D9144
:1039B000043003210693FCF721FC079A4B00D3182F
:1039C0001888DB88069A0E93089B8446D188042BBE
:1039D00008D10022B85E301AC317C018584002261A
:1039E000BB5F09E00A9B0020185E301AC6178019D9
:1039F00070400A9E1423F35EED1AEA17AD18554085
:103A0000238840190A9D059E2B806388B24AAB82A9
:103A10000C9DAB193933FF331D78002D06D0156886
:103A200062352D88A84208DC002505E0156864355C
:103A30002D88A84201DB01251D701B78002B2BD19E
:103A400012688021131C603212885E331B8800923A
:103A50004A0003F015FD069D061C0020215E002093
:103A6000285E0B1ADD175A19069B6A4094460222FB
:103A7000A55E06229A5EAD1AEA17AD185540654458
:103A8000321C2B1C05F0A6FB069B20800222A15EA7
:103A90000620185E321C78E00D9E6046B5B22B1AE7
:103AA0001BB2DA0FD3180E9A89B25B100D938B1AE2
:103AB0001BB2DE0FF3180020265E5B100896022072
:103AC000265E0E9309960D9EAB19089D1BB2EB1A4C
:103AD000DE170E9D9B1973404919099E09B2711A90
:103AE000C817091841405B180025802B01DD1D1CFB
:103AF000803D0B9803210530FCF780FB079E764B39
:103B000049001B687118039106991A1C0020085E71
:103B10005B320F99167801321278414303980B9269
:103B20000022825E0898724389180B9A42438818D3
:103B30001A1C5A3212780699104104900620095E28
:103B40000F985D334843844603981B780621415EF5
:103B500009984E430B996644414376180E991641D5
:103B60005943114176180D994B4313411A1C049B7C
:103B7000089998188022D2002B1C05F02BFB80227C
:103B80002080D2000220215E301C2B1C05F022FB7D
:103B9000514D60802B680421785E0422A15E0433BD
:103BA0003E269A5F431ADE179B19734005F012FBFD
:103BB0002B68A080F888E18804333E255A5F431AB9
:103BC000DE179B19734005F005FBE08009E000203B
:103BD0003B5EF6187610268002217B5EED186D1094
:103BE00065803C4B3C491A68059D09685319402083
:103BF0003E3118560978884203DC01225242A280E5
:103C000003E0B032116801311160483300229A702C
:103C100032E02E680599126870180692021C403234
:103C200000269657B446069E3E363678B4451CDDCF
:103C30000426B95F00291FD0483086780136F6B2D5
:103C40008670069976B23F3109788E4213DC3B8844
:103C500023807B886380BB88A380FB88E3802B68FC
:103C6000B0331A6801321A6006E00C9D059E13708D
:103C7000AA193932FF321370059D079E013D059543
:103C80000A9D0C3E023D083F0E3C07960A95F7E55B
:103C90002B680022B8331A60104B1B681C69013C6A
:103CA000611C00D197E0286862008218161C8636D5
:103CB000378805970599084F002918D09023995EF9
:103CC0008C4605990BB26146002909DC39683C3104
:103CD00008E0C04614030020581000200C03002008
:103CE00039683D3109788B4201DA0023338031880D
:103CF0000319079300293FD0983305939878844699
:103D00007F2804D001239C44059863468370079B59
:103D100098339B785BB2022B13DD90320023D05E88
:103D20003A6809B294460422944463463E229B5E5C
:103D30000593431ADA179B185340059A05F04AFA7F
:103D400030802B6802201A19111C983108563968E6
:103D500040310978884207DC211C403149005B185A
:103D600001214942D98003E0B83319680131196053
:103D700098320023D37192E73F68079B06979833E8
:103D80000227DF5705974027BC46069FBC4467467D
:103D90003F78BC46059F674518DD90321288002A9F
:103DA00000D17CE7DF79BC460127BC446746FFB2FF
:103DB000DF717FB2BC46069F41373F78BC4508DCC7
:103DC0003280B83003680133036068E7286803195C
:103DD0009833997063E711B0F0BDC04638B5041C44
:103DE0000D1C03F075F9012803D0201C291CFFF7D6
:103DF00013FC0C4B1B681A6A0023013A08D30E21EE
:103E000051436118898801395829F5D80133F4E7FD
:103E1000054A012B02DD1378013300E00023137003
:103E200038BDC0460C030020140F0020F0B58DB043
:103E3000061C0591089209930024334B1B68DB6A2A
:103E40009C425EDA2301F31808215B5E002B56D0FA
:103E5000059AA300D3180321595606919B780F1C8D
:103E60005BB20793013F069B01339F4247DC079AF1
:103E7000013A0492079B0499013399423DDC224B9D
:103E80001A687B1C91684B43049901335B180899AD
:103E9000CD5C013D2DD3D26A95422ADAAC4228D0BE
:103EA0000599A200525E12995B005B5A9A4220DC8F
:103EB000A54202DB2B1C251C1C1C210171180422AD
:103EC0000A310BA805F0E4FD290171180A310BA88D
:103ED00003F04AFF0BAA089B09990092129A0193DA
:103EE00002910392231C301C05992A1C03F05AFFEF
:103EF0002C1C049B02330493BCE70237B3E7013464
:103F00009BE70DB0F0BDC0460C030020F0B585B0B6
:103F10000C1C151C01930390FCF7D8FAFCF7E2FA8D
:103F200000F0DEFC384E3949336802201B692A1C38
:103F30004B700423CB705A230B7103F0D5F9231C6B
:103F40002A3300221A7080231B066363304BA3635D
:103F500033681A692F4B19682F4B1B6802932F4B3C
:103F600018688446013A44D3019F9600BF59A85966
:103F7000C31B676B9F4200DA6363A76B9F4200DD40
:103F8000A3630B78002B07D0029FBB18F027BF005C
:103F9000DB191B78584380110A9FBB591B0C1B1A55
:103FA00011D4487B834202DB0120664630710F202A
:103FB0000856834212DB2768181A38182060606997
:103FC000013060610AE011200856834206DCA668D1
:103FD000181A3018A060A0690130A061039F50003A
:103FE0003B52201C2A300678B34200DA331C03709F
:103FF000B8E7084B2A341B6822781B7A00209A42C3
:104000004041C0B205B0F0BD0C0300201C010020EF
:10401000FFFFFF7F4C1000205010002010030020F5
:10402000F0B595B013930C1C0C921290FCF74EFA5D
:10403000FCF758FA944B1B68FF335B79002B06D1D1
:10404000924B1B681D7A0A950A27DE5F05E0904BAC
:104050001B689D780A950427DE5F8E4D8E492B687C
:1040600002201A681B7A04324B708B7004230A708A
:10407000CB700C9A51230B71099603F035F900238C
:10408000A21D8248D3770232D3777F262968621D2A
:1040900005688248D677E21DD67700684A680F9097
:1040A0007F48013AD2B200680E920A6810907D4EA5
:1040B0008020013A000652B2AC460896079006935B
:1040C0000593002A00DAA3E00E9F50007BB20B900C
:1040D000002B00DA9AE08E68551C75430135ED1807
:1040E000A8000C9F0195139D9E00C059AE59079FD3
:1040F000861BB74200DA0796089DB54200DD089698
:10410000664637784E68002F09D0351C55430F9FFF
:10411000FF187F5D109D7843AD68684300135643D8
:104120001A9F9E19B600F659129F360C301A019E3E
:104130007500E8536646002854DB0F257557A842E2
:1041400012DB2768451B7D1925606569102701353D
:104150006561F757F67B656876B2B84201DC861B6D
:1041600000E0BE1BAE196660E568A84204DDDEB261
:10417000D7B211960D97E0606646357BA8421BDBEF
:10418000251C08351F26AE579E4200DAEB77E51D49
:104190001F26AE579E4200DDEB77A51D1F26AE57AA
:1041A000964200DAEA77651D1F26AE57964200DD7B
:1041B000EA77069F0137069785B21C9F5E0002953D
:1041C000BD5B029F7D192F1C1C9DAF531B9D0B9E39
:1041D000AF5B029EF5191B9F0B9EBD53059F3F18B9
:1041E000059711E011257557A84206DCA768451B05
:1041F0007D19A560A5690135A5612569A84200DA88
:104200002061059E361A0596013B61E7013A58E7A1
:10421000204B05981B680125D968FBF799FF2249B7
:104220007C235B42221CCB70E06176231C32281C6D
:104230000B714D7003F058F8069FA21D27621F21D5
:10424000631D51561F229A56154B1B68914201DB84
:104250001D7101E000221A71079D089EE562119F01
:10426000231C0D9D283326631F705D70E6680A9F2E
:104270000120BE4205DA2369099DD80FEA179D4245
:104280005041C0B215B0F0BD000000204C1000201D
:10429000541000200C03002048040020501000207F
:1042A00010030020FFFFFF7F1C01002007B5104B0B
:1042B0002A301B680278987C0968424392098A4236
:1042C00000DA0A1C997B4A43921101921B7B9A42A5
:1042D00000DA0193074901234B707C235B42CB70CA
:1042E00006201F2301AA0B7102F0FEFF01980EBDEC
:1042F0004C1000201C010020F0B59B4C2027A54449
:104300000F939A4B9A4C6B441B780D901593002396
:104310004B72CB7220687F230B728B720A910B92C7
:104320000323C3560F99FF1A0223C3567F00FF1AB7
:1043300049687F10FFB2089109970422815E062325
:10434000C25E0823C356407A40B20090089803F03A
:1043500097F8884B80021D682968FBF7F9FE2468EE
:104360006A682378002B00D174E0AE252D016D44DE
:104370002D68911CEB8849006B802B89AE262B8021
:1043800036010B1FEB186E441D8836687552991E56
:104390000988D9806178002903D0099D6FB27F0018
:1043A00039E0023B013A39D35E88DD88032161564A
:1043B0007519099E4D431F8871B21E89BE194E435F
:1043C0000221AD1961569E887143691889114143D4
:1043D00009141981E5E7032565575988DE886D00C2
:1043E000AC460D1CB14200D2351CADB266466E43E0
:1043F0001D89B4461E88311CAE4200D2291C0225FC
:10440000655789B29E887943754361444D19AD1152
:1044100045432D141D81023B013ADCD20F984068C0
:1044200007900B2020560422A15E0623E25E0A2399
:10443000E3560090079803F023F84E4B80021D6866
:104440006968FBF785FE4A4B2A681C682378002BB5
:104450000FD17AE0AE2109016944531C09685B0061
:10446000CB18013ADAD31988023B41430914D980A9
:10447000F7E7414D911C6D442D684900EB883E4E95
:104480006B802B896E442B800B1FEB181D883668C0
:104490007552991E0988D9806178002903D0099D39
:1044A0006FB27F0039E0023B013A39D35E88DD8884
:1044B000032161567519099E4D431F8871B21E89EB
:1044C000BE194E430221AD1961569E8871436D1885
:1044D000AD1145432D141D81E5E703256557598826
:1044E000DE886D00AC460D1CB14200D2351CADB269
:1044F000614669431E881D898C46311CAE4200D23C
:10450000291C0225655789B29E8879437543614409
:104510004D19AD1145432D141D81023B013ADCD2EA
:104520000021242216A805F0F5FA002124221FA854
:1045300005F0F0FAA22228A80021120105F0EAFAFB
:10454000237B002B1AD10F932FE00B4D531C6D448E
:104550002D685B00EB18013AE2D31988023B414316
:104560000914D980F7E7C0463CF5FFFFD80A0000E0
:10457000601000200C030020DC0A00000F9E0E22B9
:10458000A15E706800230F9388420EDD1223E3566C
:104590001025625F0093002302F072FF10231B1AA4
:1045A0009B000126119013930F96B34B00251C68B6
:1045B000109520680990099E6768721E00D2A9E0D4
:1045C000AE4E53006E443668F3181493013F00D288
:1045D0009EE00F9DA368002D3CD0099E5E43F51917
:1045E000B44601350B9E6D00705B7E1C01B2C94361
:1045F000C9170140901C58430E9530180B9D400080
:10460000455F09B20C958D4200DA0C916546EB1AB4
:10461000F3180B9E5B009B5F8B4200DA0B1C0C9D1A
:104620000B9EE8180E9BF5180223EE5E0B1EB3429C
:1046300000DA331C023DC0180026AB5F0D1E9D4200
:1046400000DA1D1C4019139E119D714368434118E7
:10465000891106E009980B9D4343FB1801335B0069
:10466000595FAE2636016E4436687B00F318149805
:104670001B890689159DCB1A9B1BAB4217DD0A9E31
:104680000B217156B94200DAF7720A9D0A21695668
:10469000B94200DDAF720A9E09217156914200DADB
:1046A00072720A9D08216956914200DD2A72991F93
:1046B000082903D816AEF15D0131F155A0680999BA
:1046C000039041431FA80C91C05D0C9D791C4D19AE
:1046D00084460B986E001295855F654500DA654645
:1046E0001FAEF555002B0DDD502B06DD002A00D145
:1046F000ACE0112A00D0ABE00023109D9D4202DA0D
:10470000109300E00023129E0D9DB1004B515DE718
:10471000099250E73D1C013D66D316ABEB5C062BBE
:10472000F9D91FABEB5C132BF5D8236828A95E1EC3
:104730000C960C9824264643AE1976006A008E1912
:104740000E925A1E0B92E6D3A2680D9853430F9314
:104750005B19191C0131890009930B580321594336
:104760000B9B89B23180002B0ED00F98831A5B19F6
:104770000D989B00C05809180D98C31858689B687D
:1047800041185918318003E00E98063128ABC15208
:10479000099B0D98990040583388C3180D9841180B
:1047A00089680C98CB180B999BB2338081420DD04D
:1047B00002314A430D99521992000D988958821876
:1047C0005B1851689268CB18D31800E00633338029
:1047D00030881421FBF76EFC0B9B3080483EB0E71D
:1047E00016ABFB5C062B02D8013FF9D215E01FABDC
:1047F000FB5C132BF8D87A0028AD236851195A1E98
:10480000F2D3A668482073435043FB180133085A7B
:104810000D9D9B005851131CF1E71949109E0A9DEC
:10482000A2682E60606826680D9D8A707C23013224
:104830005B4292004870CB70AA18832305200E704B
:104840000B7102F051FD0F4B9D44F0BD131C54E75A
:104850000C98039B0B9DC61A8E1976000398735F04
:10486000951C68430B9E08184000815F5B18D90FA8
:10487000CB185B1041E7C0460C030020DC0A0000A7
:1048800048040020C40A0000F0B500220C7D131C6F
:104890008D5C2E1BF717F6197E40012E01D0072ED6
:1048A00001D1033302E0A54201D00A33DBB2013269
:1048B000132AEDD10022632B0AD8012303700B7D4C
:1048C0001722012B04D0053B0022032B00D817220E
:1048D000101CF0BD014B18607047C046401000200E
:1048E000014B18687047C04640100020014B18600B
:1048F0007047C0463C100020014B18687047C04606
:104900003C100020014B18607047C0463810002052
:10491000014B18687047C04638100020014B1868DA
:104920007047C046140100208D23013B002B01D0AD
:10493000C046FAE7044B10221B78DBB21807C00F01
:10494000134018437047C0462B0000500F4BF7B57B
:1049500018261E700E4BA0271E70FFF7E5FFFF05FF
:104960000B4B01AC00252C3760701D703E70FFF7BB
:10497000DBFF064B20703D701D7023786278181C99
:104980005040400013400343D8B2FEBD2A000050FF
:104990002D00005010B50D4B00201B78AA2B12D112
:1049A0000B4B1C780B4B64B218780B4B40B2197848
:1049B0000A4B20181A780A4B49B21B784018801805
:1049C000C01A43425841C0B210BDC0465000020058
:1049D0005100020052000200530002005400020085
:1049E000550002008023DB020022188059809A8043
:1049F000C046024B188880B27047C04606000400CB
:104A0000154BC0229200985814490140995099586A
:104A1000FF2081434020014399509858104901409C
:104A20008020000401439950985880210002000A18
:104A300009060143995002221A6001221A600821D6
:104A400004221A601960FC3300215960054B196972
:104A50000A431A617047C04600E100E0FF00FFFF13
:104A6000FFFF00FF00ED00E013B5094A04241378AE
:104A70000021DBB21C4301910198F421FF318842EF
:104A800005DC1370C046147001990131F3E713BDC2
:104A90000D00005082B00022019201AB55221A7025
:104AA000392252429A700122DA70019AA023DB0562
:104AB0009A6102B0704700000122A023DB0510407C
:104AC0000206034998690840104398617047C04640
:104AD000FFFFFFFE82B00022019201220A408918E6
:104AE00001303F2201AB1040C9B21870481C02319E
:104AF00002408900D9705A70019AA023DB05DA615F
:104B0000196A024A0A401A6202B07047FFCFFFFFDB
:104B10000002064B000A0138002258609A60052204
:104B20001A60C0461A68D103FCD5704710E000E057
:104B3000F0B5514F85B03B6894339A7819681D7869
:104B4000DE780F231407994312092D0701922D0FC8
:104B50000B1C80222B4352001343484A0395484DB7
:104B60001340484A2B4048491340240F0B400199F9
:104B7000220413430A0545493607360F0B400096B9
:104B800013433206424E029433401343414AA02459
:104B9000E4051340E360FFF767FF3B68E268953385
:104BA0001B781540DB069B0FDB021D43E560E268C6
:104BB00080239B001343E360E26880239B0113433F
:104BC000E360029C039DFFF7E5FE002813D0324FFF
:104BD000882039781E34C9B2FBF7BAFA39784443D1
:104BE000C9B28820FBF7B4FA0F3545431E3C0023B9
:104BF0000F3D9C4203DB231E0F2B00DD0F230F22F2
:104C0000954200DD151CA024E4051F491A40E36805
:104C100012040B401343E360EB43E268DB171D40D3
:104C20000F239A431D401543E560E368F022934348
:104C300080221343E360E368144A18481340E3609A
:104C4000E3683340E360FFF763FFE26880235B05BE
:104C50001343E3600099E2680B0616401E43E660CA
:104C60000F48FFF755FF019B08491A05E3680B4001
:104C70001343E36005B0F0BD3C100020FFF9FFFFD7
:104C8000FFE7FFFFFFDFFFFFFFFFF0FFFFFF0FFF6B
:104C9000FFFFFFF0FFFFFFEF54000200FF0F0000D7
:104CA000FF6F0000064A074B12680120FC321269B0
:104CB00019789040021C0A43D2B21A707047C0465D
:104CC00014010020290000500549064B09681A7894
:104CD000FC3109690120884082431A707047C04640
:104CE0001401002029000050044B1878044B1B6865
:104CF000FC331B69184101231840704729000050FC
:104D000014010020044B82B0019001AA188092780F
:104D10009A7002B07047C0462400005007B500F0FA
:104D200069FE064B019001AA188092789A70044B94
:104D300000221A70034B0122DA7707BD24000050CD
:104D4000000F002008000050034B00221A70034B94
:104D50000122DA777047C046000F0020080000509B
:104D600072B6084B1B5C002B03D1C04662B630BF45
:104D7000F6E762B6A023DB059968034A0A409A6009
:104D80007047C046000F0020FFFFF9FF72B6074BC7
:104D90001B5C002B02D1C04662B6F7E762B6A023C7
:104DA000DB059968024A0A409A607047000F0020AC
:104DB000FFFFF9FFA023DB055A680121120E586896
:104DC0009143034A090602400A435A607047C046AD
:104DD000FFFFFFFE08B5074B1B681A1C9C321278B8
:104DE0009D331B785200013250439940FBF7B0F9D4
:104DF00008BDC0463C10002008B5044B1B689F331B
:104E0000197849000131FFF7E5FF08BD3C1000208B
:104E100008B5A0230120DB055870FFF7A1FFFFF7BD
:104E2000C9FF08BDF7B5A026041CF605042807D164
:104E3000554B1B681A1CA432A83317681B6824E062
:104E4000524B1B681A1C8C331B68883217687361BD
:104E5000FBF74EFBFB300378002B17D004F0F4FD7A
:104E600004F054FD01797F22114089040191716998
:104E70000B1C47490B400199194371614179444B1F
:104E80000A40716992040B4013437361A023DB0550
:104E90001F611E691F231E40FFF77CFD00280AD0FA
:104EA0003C4B882019780436C9B2FBF751F94643C8
:104EB0000023043E03D4331E1F2B00DD1F23A0223A
:104EC000D205108A1F210B40884303431382022C12
:104ED00016D007DC002C13D0012C2DD12B4B1D68D4
:104EE0009E3529E0042C07D023DB052C24D1264B4A
:104EF00000241D68AF351FE0234B1D68AC351BE057
:104F0000FBF7F6FA031CE0331B78002B03D01E4B93
:104F10001D685D3510E0FB300378002B05D004F0F0
:104F200093FD04F0F3FC851D06E0184B1D689B35CE
:104F300002E0164B1D68A135A023DB0559692878CE
:104F40003F22104091430143596168781F215D69F8
:104F500008401149C0022940014359610F496400CA
:104F600009680C19211C9B3108785968104091433D
:104F7000014359609C34217858680A401102084A5C
:104F800002400A435A60F7BD401000203C10002048
:104F9000FFFF03FE54000200FF07FFFF1401002083
:104FA000FFC0FFFF244BF7B51A68244B1B689E33E4
:104FB0001B785B069B0E0193131C49331978002361
:104FC0008D005519581E5B18002B27D053181B183D
:104FD0004A331B788024D3185E78A023DB055F68F2
:104FE000E4033C435C60019CB606240400945F68C3
:104FF000B60EBC46124F64462740009C27435F60B4
:10500000C046243676008400F65A2C19BC3426603B
:105010005E680C4C34405C60031CD3E7131C4933BE
:1050200009491B78BC324B700423CB700F20B0238E
:105030000B7102F059F9F7BD140100203C1000205B
:10504000FFFFC0FFFFFFBFFF1C010020F7B5FFF708
:10505000A9FF134B00241D682B1C49331E78731CB9
:105060009B005B420093B300EB180193009B043C50
:105070009C4208D0019B01211F19BC373868FFF7FB
:10508000A9FE3860F2E707492A1C0423CB70BC3222
:10509000B0230F204E700B7102F026F9F7BDC04609
:1050A000140100201C010020044B00225A70A02390
:1050B000DB055A7001221A707047C046000F0020AD
:1050C000A023DB059968064A0A40802189020A4329
:1050D0009A60044A0021917001229A707047C0467C
:1050E000FFFFF9FF000F0020024B1B68B433186864
:1050F0007047C04614010020024B1B68B43318608F
:105100007047C04614010020A023DB059868C0B298
:10511000704730B5A023DB059B68DBB283420ED01D
:1051200001DA013300E0013BA022D2059568FF219E
:105130001C1C8D430C40291C21439160EEE730BDBF
:10514000A023DB059968802252020A439A6099687D
:10515000094A0A409A609A68120112099A60D9684D
:10516000064A0A40DA60D968054A0A40DA60D96816
:10517000044A0A40DA607047FFFFFFF0FFFEFFFFBE
:10518000FFDFFFFFFFFFFFEF1B4B10B51A68012188
:10519000131C92331878A023DB059C68084017493C
:1051A0000004214001439960933210789C681449AF
:1051B0000007000921400143996011789A680909A4
:1051C0001201090712090A439A60D9688022520025
:1051D0000A43DA60D968802292010A43DA60D9680A
:1051E000802252050A43FA20DA60800000F026FC93
:1051F000FFF78EFC10BDC0463C100020FFFFFEFFF5
:10520000FFFFFFF008B50020FFF7AAFD08BD000072
:10521000034B1B689C331878400001307047C04630
:105220003C100020024B1B689D3318787047C04625
:105230003C100020004870470010005000487047A4
:10524000002000500048704700400050084B0120EB
:105250001B685B799A1C0340D318064A12689A327D
:10526000107801385843044B8000C0187047C0467E
:10527000401000201401002000400050074B012086
:105280001B685B799A1C0340D318054A12688A325E
:1052900010785843034B8000C0187047401000201E
:1052A0001401002004400050F7B5264B051C1C6873
:1052B000A3795F1E15D36279013A10D36079561C29
:1052C000811C0191012108400199081858433118A7
:1052D0001D48890009180868E8400860ECE73B1C95
:1052E000E7E714220A23013B0ED360790121871CD2
:1052F0000840381850435E1C3118134889000918BB
:105300000868E8400860EEE70132162AEAD1FFF7A4
:10531000B5FFA37A002201339C466346013B9C46BD
:105320000FD3617A96000191861900230199994261
:1053300005D09F00F1590133E940F151F6E75218C9
:10534000EBE7F7BD4010002000400050074B012064
:105350001B685B799A1C0340D318054A1268963281
:1053600010785843034B8000C0187047401000204D
:105370001401002004400050094B01211A685379A0
:10538000D0799A1C0B40D318064A013012688E322D
:1053900012785343C018044B8000C0187047C046B1
:1053A000401000201401002000400050F7B5434B8E
:1053B0001D682A7853B2042B1DD1414B19680B1C70
:1053C000AE331F7802235E1E77D34A79013A10D399
:1053D0004C79551CA01C019001200440019804192F
:1053E0005C432819374C800000190468FC400460B5
:1053F000ECE7331CE7E7002A45D0022B21D1FBF76D
:1054000077F8E03003782E4C002B02D023685F330E
:1054100002E02D4B1B689D331878FFF745FF256888
:10542000EC79002C2FD0FFF7A7FF061C013C2AD3F4
:10543000697A201CFAF7E2FE89008A59A300F2502B
:10544000F4E7032B03D1204B1B68A33318E0012B97
:1054500011D1FFF77BFF1A4B061C1B685C79013CDE
:1054600011D32B195E331B789B009859FFF7C4FCAE
:10547000A300F050F3E7052B05D1114B1B68B133A6
:105480001878FFF711FF104B1B689A331B78002B1D
:1054900013D00B4B1A685379013B0ED35179012578
:1054A0008C1C294061189479581C614340180549A7
:1054B0008000401800210160EEE7F7BD14010020D4
:1054C00040100020004000503C10002008B5A023F0
:1054D0000120DB055870FFF743FCFFF76BFCFFF77B
:1054E00065FF08BD70B5041C104E114D11D101208F
:1054F000FFF798FC336801221A70A023DB056C705B
:105500005C701A70FFF7E2FFFFF754FCFFF79EFD97
:105510000224201CFFF786FC336800221C70A023A5
:10552000DB056A705A7001221A7070BD14010020E8
:10553000000F002008B5FFF7D5FFFFF7C7FF08BD34
:1055400010B5A023DB051C6A0005064A000D010406
:1055500022400A431A621A6A120B1203104318629D
:1055600010BDC046FFFF00F073B5174BA0221B68AB
:10557000D20590339168196891601C78FFF70AFA98
:10558000124D002812D0124B124A1B7812782E6846
:1055900052B25BB20092201C1021D12201F070FFA8
:1055A0002B68B8363060B8331B68E418002C01DA79
:1055B000002402E0FF2C00DDFF242B68E0B2B433AE
:1055C0001C60FFF7A6FD73BD3C10002014010020F5
:1055D000530002005200020073B5154B1B683233B2
:1055E0001C78FFF7D7F9134D002812D0124B134A3D
:1055F0001B7812782E6852B25BB20092201C1021E8
:10560000D12201F03DFF2B68B8363060B8331B68FB
:10561000E418002C01DA002402E0FF2C00DDFF2456
:105620002B68E0B2B4331C60FFF773FD73BDC04656
:105630000C0F002014010020530002005200020051
:1056400008B5002801D0012801D100F09DFEFFF728
:105650008BFFFFF76DFAFFF71DFA08BD70B51F4B02
:1056600013211B68A0B0DA7A0023133AD2B2914218
:105670005B410221C91AA023DB0558693F22104073
:105680005C688022D20322435A60421EA023D2B219
:10569000DB05FF2A11D05E683F25114C15402D0413
:1056A00034402C435C60C0460C1C243464001C5BFA
:1056B0006D465300EC52013AE8E75968094A0A403E
:1056C00009495A6002234870CB700320B3236A460D
:1056D0000B7101F009FE20B070BDC04640100020E3
:1056E000FFFFC0FFFFFFBFFF1C010020F7B5041C38
:1056F00002F05EFA124B1A6800235068411C0191B7
:10570000019D16689D420CDB976801367E43990027
:105710008C469E1900216546B60061510133315116
:10572000EEE701239E420ADB956800215D43AF004E
:105730002D180135AD00395101332951F2E7F7BD7C
:105740000C030020044B054900221A6059609A603E
:1057500005221A607047C04610E000E0FFFFFF001E
:1057600010B5A023DB059C6899680C4BC9B21B6877
:10577000E403B8331B68E40F591AFF31E623594399
:105780000134074BA040C918041C0648FAF7E0FC96
:10579000C1B2201CFAF7DCFC10BDC0461401002089
:1057A0005C5D000040420F00014B00221A60704710
:1057B00010E000E013B50B4C0B48A368C01A01932E
:1057C000FFF7CEFF094901234B7004230190CB70F2
:1057D00000206F2301AA0B7101F086FD00230198C0
:1057E000236016BD10E000E0FFFFFF001C01002059
:1057F00010B5041CFFF7A6FF201CFFF773FEA023C3
:10580000DB0501205870FFF7C1FAFFF7D3FAFFF765
:10581000CDFDFFF7CFFF10BDF7B51F4800F00EF923
:10582000FFF776F91D4B00251C1C1D4EB34216D206
:105830008036F61A2020832E00DCB01080101A1C4F
:10584000011C013908D3002D04D1164E1768B74248
:1058500000D0151C0432F4E780001B18E5E72B1B71
:10586000114C019304230127E370211CA72301AAF3
:1058700000208436751B67702371042601F034FD07
:10588000A8230020211C01AA01956770E6702371EE
:1058900001F02AFDF7BDC046801A060068100020FE
:1058A00080370020CDCDCDCD1C010020024B1B68E0
:1058B000493318787047C0461401002070B5051CA4
:1058C000FFF744FD0B4B1C68231C49331B789A00DF
:1058D000AD180022511ED218002A09D0E218521821
:1058E0004A321278920016588A00AE500A1CF1E72C
:1058F00070BDC046140100200B4B30B51B681A1C4C
:105900004932127894001C195300C0180023013347
:10591000D11A013107D09D00651BBC3559002D6897
:1059200049424552F3E730BD14010020F8B50C1C84
:10593000051CFEF7EDFF144908688379013B11D37C
:105940000E687279013AF9D30E6870790F4E584398
:1059500036688018F6182818A03607783679BE19E8
:105960000670EFE70B68DB79013B08D3074AE15C7F
:105970001268D218C83212788A18E254F4E7281C48
:10598000211C00F05FFCF8BD401000203C100020FE
:10599000134BF7B51C686946E26800AF131C0E3361
:1059A000DB08DB00C91A23698D460E33DB08DB00F8
:1059B000C91A0C4B6D461E688D467960281C311C37
:1059C00004F066F8F0239B00F1182269786804F06F
:1059D0005FF8281C7968FFF7A9FFBD46F7BDC046F0
:1059E0000C03002038100020A023DB0518690006F6
:1059F000400F704738B5A023DB0599689D680C4BB4
:105A0000041C1B680B48B8331B68ED03C91AC94353
:105A1000E623C9B25943084BED0FC918FAF798FBB2
:105A2000044B01355843211C2841FAF791FB38BD3E
:105A30001401002040420F005C5D000038B5A02337
:105A4000DB0599689C680A4B051C1B680948B8333C
:105A50001B68E403C91AC943E623C9B25943064B7C
:105A6000E40FC918FAF774FB68430134204138BDCC
:105A70001401002040420F005C5D0000002801D0AE
:105A8000133907E0122902DD262902DD12394910F7
:105A900000E000E0081C7047F0B5AA4B00261D6826
:105AA000041CEB7A1322133BDBB2301C9A42704188
:105AB000B1B0C7B2059702273F1A311C142209A8BA
:105AC00004F028F8A04B20681B68882201938F33CC
:105AD0001870019B6168923319700EA8311C04F094
:105AE00019F8311C142209A804F014F8974B0EA8D9
:105AF0001968442203F0CCFF022F04D11FA80EA97D
:105B0000442203F0C5FF00272E1C0497771B039740
:105B10006B7901369F423EDAB77A0598391CFFF758
:105B2000ADFF09A9095C0EAB0291029A44215143D1
:105B300009185918721B0A717911069109A90A5C92
:105B400011214A43069952181F210F4006320121A4
:105B50009200B9400F1CD1580F43D7500399019FB1
:105B60003F237A185178071C99438C4602991F40AD
:105B700089010691614603970F431F40069B1F430F
:105B8000029B5770013309AFDBB23B54049F9F4225
:105B9000BCDA0493BAE7019B049D913300261D7083
:105BA0000296684B029E19688F79BE4200DBBEE008
:105BB000029D49190B1C2833DA79644B1E68331C8B
:105BC0009A331B78B446039303980023984204D079
:105BD000781E854201DA2931CB790120011C9140E0
:105BE0000591111C2039051C8D40A9011D1C203D6B
:105BF000061CA840049D9E408909069607900195C1
:105C0000019D002D38D0019E4425013E754301962B
:105C100066680EA82E544519281C002620302E62D6
:105C20004668B60EB606009646601F2A02DC059846
:105C3000286204E08D01009EAD092E434660039D5D
:105C4000002DDDD0029E781E8642D9DA019E4425C1
:105C500075430EA845191F2B04DC2E6A06983043A5
:105C60002862CDE7686A079E0643B601800EB60932
:105C7000800630436862C3E7029E6046331C457865
:105C80006344C833AD065F79AD0EFEF783FE00288E
:105C900013D02F4E882031780137C9B2FAF758FA5D
:105CA00031784743C9B28820FAF752FA02354543A2
:105CB000013F023D019E791C03D03E1E1F2E00DDD8
:105CC0001F263F2D01DD3F2526E0EB43DB171D405E
:105CD00022E00199442251430EAB59188F781F23BB
:105CE0009F43301C18403B1C03434F788B703F236D
:105CF000281C9F4318403B1C034320684B703B28E3
:105D00001CDC5043134FC01903F0C2FE2368019FEF
:105D10000133013723600197019F04988742D8DB44
:105D2000029D6368013501330295636039E7064BD4
:105D300022681B68012090331A7000E0002031B007
:105D4000F0BDC04640100020140100203C1000208F
:105D50005400020000800050124B30B512491B68FD
:105D6000002810D00A2209685A6048790125841C4D
:105D700028402018986089799A611960514314224B
:105D8000D960DA610CE00A680125517959605079CF
:105D9000841C28402018986092791A604A43DA607F
:105DA00030BDC0460C0300204010002030B5074B2A
:105DB00085B01B6801A8021CA83332CB32C2FFF7A2
:105DC0006BFEFFF7E5FD05B030BDC04614010020B5
:105DD000F0B5574B9FB01B6800270493DB7A132262
:105DE000133BDBB2391C9A427941CBB2051C391CFA
:105DF000142208A8079303F08DFE4E4B2A681E68F4
:105E00000DAC331C93331A706968023359701F70DC
:105E1000391C4422201C03F07DFE391C142208A8E2
:105E200003F078FE444B201C1B684422191C069387
:105E300003F02EFE331C49331F70049A53799F429E
:105E400034DA049A0798D319DB7A191C0593FFF703
:105E500015FE08AB1B5C9C46002B0CD1331C493350
:105E60001A78511CB21819704832FBB20DA9937000
:105E700001330A1813710DAB19180979F2195E3242
:105E800001391170059901374A11063292000392C7
:105E90001F220A4001219140039AD2581143039ACC
:105EA000D1506346013308A90B54C6E7069B5E78C0
:105EB000B606B60EFEF76EFD00280AD01F4B8820EE
:105EC00019780236C9B2FAF743F946430023023E75
:105ED00003D4331E3F2B00DD3F23A2781F218A43CA
:105EE0006178A2703F2291431340626A0B43696854
:105EF0006370930E21709B06002119A81422216261
:105F0000636203F007FE2868442250430C4B211CB7
:105F1000C01803F0BDFD6A682B6801326A60054A4B
:105F200001331268012094322B6013701FB0F0BD52
:105F300040100020140100203C10002054000200FA
:105F400000800050F0B5BA4BB1B01B680024039339
:105F500053331B78071C133BDBB21322201C9A42DD
:105F60006041C5B2059502252D1A211C142209A8ED
:105F700003F0D0FDAF4B3E681B68211C04938733B0
:105F80001E70049B78688A33187088220EA803F06C
:105F9000C1FD211C142209A803F0BCFDA64B0EA8CC
:105FA00019684422443103F073FD022D04D11FA867
:105FB0000EA9442203F06CFD0025039C0695039E68
:105FC000039DA61B07966B7A01349E4237DA231C89
:105FD00052331D780598291CFFF750FD09AA115C62
:105FE0006E118C460296112166467143029E0EABDD
:105FF00089191F263540063101268900AE40351C1F
:10600000CE583543CD50079E049D3F23A919051C4A
:106010001D40803166460295B6018D780196029E3C
:106020009D432E431E40019B069D1E436346013344
:10603000DBB28E7013549D42C1DA0693BFE7069E11
:10604000049BF6B2893307961E700024784B0494A3
:106050001B68049D9A7A954200DB9BE0049D069C98
:106060005A19583211780122081C2038161C824017
:106070008E409001B44680090394039C002C1BD0F1
:10608000039D4422013D6A437E680EAC1655A2185A
:106090000395141C1F2905DC566A65461562B20E6D
:1060A000920607E000251562666A8201B50E920924
:1060B000AD062A436262E0E75E4A1168221C587A04
:1060C000824210DA8818803084784425A006A4091A
:1060D0006C43BE68800E20180EAD0136281806717C
:1060E0000132BE60EBE7544B1B681A1C4632453345
:1060F00016781C78F606A406F60EA40EFEF74AFCE7
:10610000002813D04D4D882029780136C9B2FAF7FE
:106110001FF829784643C9B28820FAF719F80234E3
:106120004443013E023C0025701C03D0351E1F2D48
:1061300000DD1F253F2C01DD3F2402E0E343DB1798
:106140001C40039E0698864221DA0399442251435B
:106150000EAB59188E781F239E43281C1840331C01
:1061600003434E788B703F239E43201C1840331C02
:1061700003433868324E50434B70801903F088FC5B
:106180003B68039E013301363B600396D9E7049CCC
:1061900001345BE7274A3E681468079D221C883259
:1061A00016703868D0707968053251701570002209
:1061B000597A8A4210DAA1188031897844208D06F4
:1061C00089094843AD0EB96840190EAE0131301847
:1061D00001710132B960EBE71AAD03950025069E07
:1061E000B5421EDA44236B430EA8C618706A00211C
:1061F000820E9206316272620398142203F08AFCC6
:106200003868442148430E4A311C8018442203F068
:106210003FFC3B68039E013344363B6001350396E7
:10622000DDE73B688C340120237031B0F0BDC046FF
:1062300040100020140100203C10002054000200F7
:1062400000800050F0B5374B85B01B6802901A1CD7
:10625000039187321578344A00201168041C8A7A29
:1062600094422BDA021C4F7A161ABE421FDA9E198C
:106270008036B678B7090096EF1944267E432B4F37
:10628000B4463E1C009F66440196BE06039FB60EB0
:10629000B446BE5C3F2E00DD3F26F6B20096019E5E
:1062A0000132371C6744009E30373E70DBE7181C14
:1062B0008930007801342D18101CD0E71A1C8F3259
:1062C000147800208A79904229DA00224D790195CC
:1062D000AA421EDA9E187678B709E7190397442771
:1062E0003D1C039FB6067D43AC46104DB60E2F1CD9
:1062F000019D674445430397029FBF187D5D3F2D75
:1063000000DD3F25039FEDB2BE19303635700132F6
:10631000DCE71A1C913212780130A418D2E705B0DC
:10632000F0BDC04614010020401000200080005045
:10633000134BF0B5196800220B1C97331C7800230F
:10634000CD1820356D794426AF09E71977430D4EF6
:10635000BF19AE068518ED5CB60E3F2D00DD3F255A
:10636000BE19EDB23036013335700A2BE8D10B1C63
:1063700099331B780A32E418142AE0D1F0BDC046E4
:106380001401002000800050F0B5CD4B00251C68A2
:106390002F1CE27A1323133AD2B2B9B093426F4161
:1063A0000223DB1B291C0C2209A8019303F0B2FB7A
:1063B0000CA8291C142203F0ADFB6679FFB20296EB
:1063C000261C029A331B934214DAF17A381CFFF729
:1063D00055FB132801D9002002E20CAA135C019995
:1063E00001368B42F7DA0133DBB213549D42E8DA0F
:1063F0001D1CE6E701220992A079002181420ADAF8
:10640000131C9E1AAE4203DA3B2BE4DC0133F8E79F
:1064100001311A1CF2E70992E379002B35D10025EE
:1064200009A80995FFF7D4FC09A8FFF735FBA44E8E
:10643000A44A346812680998E67A0192973210707B
:106440000A9B019A01339A32133E1370291C882249
:10645000F6B2132716A80A93B742BF4103F05AFBBE
:10646000291C142211A803F055FB7F42211C01377F
:10647000603116A8442203F00BFB022F40D127A85D
:1064800016A9442203F004FB3AE0231C53331B7883
:106490000025133BDBB21322291C9A4269410222D8
:1064A000521A0192CFB20CA8291C142203F032FB1D
:1064B000667A0296261C029A331B934215DA331C25
:1064C00053331978381CFFF7D9FA132883D80CAA4C
:1064D000135C019901368B4200DB7CE70133DBB2B0
:1064E00013549D42E7DA1D1CE5E7EB43DB171D4023
:1064F000A37A5D43099B6D00ED183B2D8FDD6AE7A4
:10650000231CA11D621D2F330B34132E04D80591BB
:1065100004920693039403E0049105920393069476
:10652000002402940424049E3378043B9C4234DA11
:10653000039E0120355D11AF291CFFF79FFA3A5CDD
:106540004426564316AB36189E19E11E31713E5C47
:1065500011277E43691171181F2635400631012627
:106560008900AE40351CCE58019F3543CD503919B6
:106570001C314F793F23061C1E409F433E4395012B
:106580001E402E430132029D4E71D2B211A90A540F
:10659000954200DA02920134C5E7019B029F9933CC
:1065A000059C1F702378043B0193059D019E2B7869
:1065B0009E4200DBB7E0069D019E0A9FAB19013B9E
:1065C000A95D187801231A1C8A40FFB204920A1CA4
:1065D0001C1C0397203A071C94401D1C203F079465
:1065E0008540BB40029CAC461F1C002C37D0013CB0
:1065F00044236343039E16AA9E54D3181A1C0025F5
:106600001D6220325668B50EAD065560DD78202635
:106610003543DD701F2904DC1D6A049A2A431A627F
:1066200008E05368079D1D43AD019B0EAD099B0615
:106630002B4353604422624316AEB2181F2804DC79
:10664000156A63462B431362CFE7536A1D1C3D4313
:10665000AD019B0EAD099B062B435362C5E71A4B58
:10666000019F1B68DB19C8335F79154B1B686133C9
:106670001D78AD06AD0EFEF78DF9002813D0134E30
:10668000882031780137C9B2F9F762FD3178474384
:10669000C9B28820F9F75CFD02354543013F023D50
:1066A000261C781C03D03E1E1F2E00DD1F263F2D0A
:1066B00001DD3F252DE0EB43DB171D4029E0C046FF
:1066C00040100020140100203C1000205400020063
:1066D0004422111C614316AB59188F781F239F4326
:1066E000301C18403B1C03434F788B703F239F4363
:1066F000281C18403B1C099F03434B703B2F1FDC99
:10670000101C7843374B0137C01803F0C1F901342E
:106710000997029FBC42DBDB019C0A9B02340133D8
:1067200001940A9341E7304B099F1B6816A89833E0
:106730001F702E49142203F0ABF916A8FFF7F8FDDD
:10674000294C2068021C9832031C127890331A706E
:10675000274B1B68DD79002D03D009A8FFF7F2FB5A
:1067600014E0291C0422873003F0D4F92068291C86
:1067700004228B3003F0CEF923680998191CC2B2A9
:1067800087318C330A704A700A711A702468231C8E
:1067900093331A78073BDA73211C1B789C310B70FA
:1067A0004A7008390978221C9E3211700F3A157808
:1067B000211C9F31201C0D70A1305374022203F064
:1067C00067F9231C97331B78221CA3321370023302
:1067D0005370231CA8331D609234227801205A6024
:1067E00039B0F0BD0080005014010020DE9F000091
:1067F00040100020F0B5B5B0A749142208A803F056
:1068000047F9A64B00261D6813222B1CA8331B68D2
:10681000301C05932B1CAC331B68311C0493A04B1C
:106820001C68E37A133BDBB29A427041C7B2069709
:1068300002273F1A2B1C0598973301221870DA7033
:1068400012A8882203F066F9311C14220DA803F067
:1068500061F9211C603112A8442203F019F9022FBA
:1068600004D123A812A9442203F012F90027261C00
:106870000397371B0297637901369F423DDAB77A57
:106880000698391CFFF7FAF80DA9095C12AB0191C3
:10689000019A4421514309185918321B0A71791180
:1068A0000DAA0791115C11225143079A89188A1D7C
:1068B0001F210F4001219200B9400F1CD1580F43F6
:1068C000D750029F3F23EA19011C019F2032194033
:1068D0000291BF0151790797029F99430F4307998E
:1068E0001F40019B0F4357710133039FDBB20DAA79
:1068F00013549F42BDDA0393BBE7039E99352E7074
:10690000A379043B0193664B019F19688B799F42E1
:1069100000DBB1E0019FCB191A1C28320F33D0796C
:10692000DC7F01231A1C82400292021C203A1D1CAB
:106930009540221C1E1C203A0695A6409340039DBC
:1069400007969C46002D37D0013D44236B43049F9E
:1069500012AA9F54D3181A1C00261E6220325768B0
:10696000BE0EB6065660DE7820273E43DE701F2836
:1069700004DC1E6A029A32431A6208E05368069EDB
:106980001E43B6019B0EB6099B0633435360442257
:106990006A4312AFBA181F2C04DC166A079B3343F4
:1069A0001362CFE7536A66461E43B6019B0EB609D3
:1069B0009B0633435362C5E73A4B019E1B68613126
:1069C0000C789B19C833A4065E79A40EFDF7E2FF8C
:1069D000002812D0344F882039780136C9B2F9F72F
:1069E000B7FB39784643C9B28820F9F7B1FB0234C6
:1069F0004443013E023C771C03D0351E1F2D00DDB1
:106A00001F253F2C02DD3F26029603E0E343DB1700
:106A10001C400294059E442777432448341C3F18A9
:106A2000039AA11B059491421FDA4422514312ABF1
:106A30005918281C1F231840059088789843031C78
:106A4000059803438B7002983F23184005904878BF
:106A50009843031C059803434B703B2C17DC381CF0
:106A600003F016F801344437DAE7019D049E02353D
:106A700001360195049646E7084B059D1B680121E8
:106A80001A1C98321570D172A43303221A7008A808
:106A9000FFF74EFC35B0F0BDDE9F00001401002072
:106AA000401000203C1000205400020000800050E4
:106AB00030B50F4B1B689979884203DA1B182833CD
:106AC000D87914E05A798D18411AA84202DA5B1875
:106AD000D87A0CE09C7A8A1A2D19A84203DA9B18FE
:106AE0005833187803E0141B1B195033D87830BD85
:106AF00040100020F0B5D44DA024E405A3682B6815
:106B000097B059799A7900AF8A18597A9B7A5218B6
:106B1000D3181A1C5A437B62D31DDB08DB0068467E
:106B2000C01A85466B46FF217B6102F0F3FFFF2010
:106B3000FEF784FFC54B69461B1A786ABB60C0002C
:106B4000031C0E33DB08DB003861C91A786A8D46F6
:106B50006B4680003B62031C0A33DB08DB00C91A6A
:106B6000002200233A637B63F860F961E268B84B66
:106B70008D461340E3602B685C79B34B013C1B6886
:106B8000621C14D01B19381CD97A5030202202F014
:106B900061FF3D6D58207A6DAB00C019C31801210B
:106BA000283B91400A1C19680A431A60E5E79C7962
:106BB000A54B013C1B68621C15D01B192833381CDF
:106BC000D9795030202202F045FF3D6D58207A6D72
:106BD000AB00C019C3180121283B91400A1C196859
:106BE0000A431A60E4E75C7A974B013C1B68621C1D
:106BF00015D01B195033381CD9785030202202F0A0
:106C000029FF3D6D58207A6DAB00C019C3180121D2
:106C1000283B91400A1C19680A431A60E4E79C7AF1
:106C2000013C621C17D0884B381C1B6850301B1964
:106C300058331978202202F00DFF3D6D58207A6DEF
:106C4000AB00C019C3180121283B91400A1C1968E8
:106C50000A431A60E4E77D69BD610025FD62FD6AB3
:106C6000786A854200DBDEE000213A69386A02F08A
:106C700051FFA0240021FA68F86902F04BFFE405F7
:106C800000232363636B9B0E9B0663633D6BA563CD
:106C9000786BB862E36B86019B0EB6099B063343A3
:106CA000E3636420FEF7CAFEFDF732FFF86AFFF7E0
:106CB000FFFEC1B2381C4830202202F0CBFE396BF7
:106CC0007A6BFB6CB963FA63BA6C01219940582066
:106CD0000B1CC01991004118081C203802689A4307
:106CE0000260B86C131C00280AD028390A68534087
:106CF0009A01636B92099B0E9B061343636301E049
:106D00006B402363A024E405A563E36B0A209B0E7C
:106D10009B061E43E663FEF791FEFDF7F9FEE26B6C
:106D20008023DB041343E363B96BBA6A4D40A56368
:106D3000FB6B5A40E36B92019B0E92099B06134337
:106D4000E363FEF7FFFCFD6BBE6B3B6AAC460124C0
:106D5000404ABD689168A94214DB3F4A6546106805
:106D6000526830402A405D68954203D3F0D11D68D7
:106D70008542EDD2FD69DA60A2009860A950013425
:106D80000833E5E7FEF710FDA023DB05D96B334A96
:106D90000A40DA63012C3ED0651E386AED004519C1
:106DA000013C002C37D02B1C083B1A6829685B6813
:106DB00091436A687E6A9A43A30039647A64013E0B
:106DC000BB62FA6A964224D0301CFFF771FE011CA8
:106DD000381C5030202202F03DFE7B6D0122386DC0
:106DE0009A405821131CC91982008A18183A12684F
:106DF0001A420CD0BB6AFA691720D258404250435D
:106E0000174BC018FEF7ACFCB96900118855013E5C
:106E1000D7E7083DC4E7FD6A786A0135FD62BD69C0
:106E20002D18BD611BE7C3B2381C5030037043708E
:106E300083700023C370037179690123437100F0EB
:106E400097F9BD4617B0F0BD40100020FFFFFF00CE
:106E5000FFFF0FFF10E000E040000050FFFFFFFBCE
:106E6000E9FFFF16014B18607047C046481000202C
:106E7000014B18607047C04644100020F8B5F9F780
:106E800025FB071C00F094FE061CFDF729FD2D4D87
:106E90001022041C391C286802F0FAFD32882B6885
:106EA0001A74120A5A74B2889A74120ADA74264A48
:106EB00012680532D27F002A03D0A2791A7562794E
:106EC00002E062791A75A2795A75E2791F4C9A75B7
:106ED000231C0833AB60A0236C60DB056E69DB7C90
:106EE0003370FDF733FD627E217E12020A43A17EDC
:106EF000F07109040A43E17EEB6809060A43110AAE
:106F00001A705970110C120EDA70627F9970217F1D
:106F100012020A43A17F09040A43E17F09060A43DA
:106F2000110A1A715971110C120EDA71221C2C32CD
:106F30002D3499711178227812020A431A72120ABA
:106F40005A72F8BD2C0100200C030020D0BF0000B5
:106F5000F7B5F9F7BBFA051C00F02AFEFDF7C0FCF7
:106F6000144CAA6BE369A56A59685A6002F0ACFC3C
:106F70006860FFF783FF104B226B1B680F4819886E
:106F80006D460B0A11715371C0C8C0C589006B46AC
:106F9000CB589371231C3C3301225A7000229A7003
:106FA00002F08CFC064B5860A023DB059A7C236C16
:106FB0001A70F7BD2C01002048100020F49F00003B
:106FC0005804002008B5084AD1694B780749DBB25C
:106FD0000B72012B05D0022B05D1936901225A7047
:106FE00001E0FDF75FFE08BD2C01002058040020E1
:106FF000094B10B51B7A094C012B05D0022B05D18A
:10700000A2690023537001E0FDF75EFE636B7F21F0
:107010001A788A431A7010BD580400202C010020F1
:10702000F8B5194D0024194E337A012B07D0002BE7
:1070300018D0022B17D1164B9B695C7813E0FDF733
:1070400053FE041C002D0BD1FDF73EFE2E23FF3313
:10705000013B002B01D0C046FAE7FDF723FE0A4DA5
:10706000013D00E01C1C0A4FFA695378327A9A42BB
:1070700006D0FFF7BDFFFB69044A5B78137201E09D
:10708000002CD0D1F8BDC046FF2C010058040020D0
:107090002C010020024BDB691878C0B27047C04653
:1070A0002C010020024BDB695878C0B27047C04603
:1070B0002C010020024BDB699878C0B27047C046B3
:1070C0002C010020014BDB69987070472C010020D7
:1070D000024BDB69D878C0B27047C0462C01002053
:1070E000014BDB69586870472C010020024BDB69BB
:1070F000187AC0B27047C0462C010020024BDB69F1
:10710000587AC0B27047C0462C010020024BDB69A0
:10711000D87AC0B27047C0462C010020024BDB6910
:10712000987AC0B27047C0462C010020024BDB6940
:10713000587BC0B27047C0462C010020024BDB696F
:10714000187CC0B27047C0462C010020034BA0221F
:107150009B691A701A78A02AFCD070472C01002075
:10716000024B9B6C1878C0B27047C0462C010020BF
:107170000E4B30B59A6CFF2414700D4CD86421600E
:1071800005788478996A6C430579407964194006DA
:10719000400E604308609869A0210170D969137896
:1071A000FF2B02D10B78022BF9D030BD2C0100202F
:1071B00058040020014B1B681888704748100020B5
:1071C00008B5FFF72DFF024B0022DA6008BDC0466C
:1071D0005804002070B5074B074C1A6BE668011C79
:1071E0009579986B2A1C8019751902F051FCE5609D
:1071F00070BDC0462C0100205804002008B5074B84
:10720000DB68002B09D0064ADBB2506B7F211940A6
:1072100001703C329370FFF7D5FE08BD5804002082
:107220002C010020F8B5071C0E1CFFF7F9FE0D4CD1
:107230008020636B40421978F6B208437F22C0B2C7
:107240009043311C1140021C0A43A56BA7631A70BE
:10725000231C3C339E70FFF7B5FEFFF7E1FEA563EC
:10726000F8BDC0462C010020014B5B6D18707047C3
:107270002C01002073B56C46E271194A0734556D34
:107280002E7886422AD1FF2028701366131C94336F
:107290001B6820789B6880009165D4651871114B3C
:1072A00006980C7818608878936A60430C7949795D
:1072B00000194906490E414319609169A0230B70DA
:1072C000516DD3690A78FF2A02D11A78002AF9D0C1
:1072D0000A78FF2A02D11A780A2AF3D073BDC04671
:1072E0002C0100205804002070B5144C636B1D79EC
:1072F000EDB2012D21D1854058781E78000230432F
:107300009E7836043043DE7836063043284214D067
:10731000FF2018710A48A16302608C780D78C97843
:107320006C434906490E074A6143906A92690160BD
:10733000772111701A79FF2AFCD070BDAC010020B2
:10734000580400202C010020014BDB6B187870479B
:10735000AC010020014BDB6B18707047AC010020C2
:10736000014BDB6B58787047AC010020014BDB6BA5
:1073700058707047AC010020014BDB6B9878704768
:10738000AC010020014BDB6B98707047AC01002012
:10739000014BDB6B18797047AC010020024BDB68B6
:1073A0009872000AD87270472C010020024B5B696A
:1073B0001872000A587270472C010020024B5B695A
:1073C0009872000AD87270472C01002000230360D5
:1073D0000B601B4BF7B59A4230DC1312194C122B81
:1073E0001BD89B00E418646E002C27D0E368013B97
:1073F0005D1C23D0D5B2019565681E1CEF5C019D14
:10740000013BED1BF4D42768B300DB59002B15D0EA
:107410005B190360A3689B5D0EE0E36A666A013B4B
:107420000CD35D00755B551BF9D4266A9B00F2589E
:1074300052190260A26AD3585D1B0D60F7BDC046A9
:10744000FFEF00002C010020C02208B5D2000B4B3A
:10745000904206D19B691A78052A0DD005221A7030
:107460000AE05B6B84221B7892005B065B0E9B1824
:10747000984201D1FFF7BCFD08BDC0462C01002099
:1074800038B5051C1C1C181C8D4209DB049895425C
:1074900006DAC01A6D1A6843511AF8F759FE201817
:1074A00038BDF8B501254E1E6C00B54202DA165FF4
:1074B000B0420CDAA61E1D5F115F9B5F401AEB1AEB
:1074C0005843935FC91AF8F743FE4019F8BD0135D8
:1074D000E9E70000014B18607047C04654100020D7
:1074E000014B18687047C04654100020014B1860CB
:1074F0007047C0464C100020014B18687047C046CA
:107500004C100020014B18607047C04650100020FE
:10751000014B18687047C04610030020F0B5041CEA
:1075200087B000200D1C2C4902920393021C4F23AC
:107530000B71FFF7D9FE294B00201A685368013BF5
:107540000FD399006F5811684E1EB446F7D3966852
:1075500071435918013189000959C91B4018614606
:10756000F2E7D168F8F7F4FD1D4B071C1D681D4CB0
:107570006E88002E03D1236840229A600CE0A9880F
:107580002268701A8001791A0192F8F7E1FD6E28DD
:1075900000DD6E20019B9860AB7964225343029A10
:1075A0005343039A13412A78002A03D02268926831
:1075B00053439B1122680C49D36002234B707C23F8
:1075C0005B42CB700020502304AA049605970B71F0
:1075D000FFF78AFE07B0F0BD4F0400200C03002027
:1075E0004C100020100300201C010020F0B585B0D5
:1075F00001912449D2690968051CC9798A40002A89
:1076000000DC012220490968C868191C5043F8F7BA
:107610009FFD1E4B02901C6820680390021C571EA1
:107620001AD36368191C7943C91889006918043989
:10763000013B0FD3A66801205643B4469C448444C2
:10764000664686400198305E029E46430868801B6D
:107650000860ECE73A1CE2E70D4E1023B371039B80
:10766000042033702379311C7370B3702A1C60239B
:10767000F0703371FFF738FE00230120B37105B0BD
:10768000F0BDC0464C100020100300200C03002069
:1076900048040020F8B5144B051C1B680E1CD86864
:1076A000111CF8F755FD114B1B681A6994002C1931
:1076B000131C043C013B06D35900715E276841430B
:1076C000791A2160F5E70A4C1023A3716270042037
:1076D00061232A1C211CE0702371FFF705FE0023A3
:1076E0000120A371F8BDC046100300200C03002048
:1076F0001C010020F0B585B003931A4B00901C6864
:107700000291256801926F1E1BD3636800981E1CAE
:107710007E43F618B6008619043E013B0FD3A168DC
:10772000012269438C469C44944460460199800040
:10773000425830689446844461463160ECE73D1C11
:10774000E1E72269039D029C9300E118E8180023F9
:10775000043B013A04D3CE58C5587419CC50F7E70E
:1077600005B0F0BD0C030020F8B5061C58780D1CC0
:10777000400091780130884051789B784900013170
:1077800099408003F8F7E4FC1349041C0020B4235B
:10779000021C0B71FFF7A8FD104B18680268013A34
:1077A0000DD34368191C5143C91889007118043955
:1077B000013BF4D30F68BF0B67430F60F7E7036922
:1077C000990069180439013B04D30868820B6243AD
:1077D0000A60F7E7F8BDC0464F0400200C03002004
:1077E000F8B5051C50788B784000497801309840F6
:1077F00049009378013199408003F8F7A9FC0E49BC
:10780000041C0020B423021C0B71FFF76DFD0B4B11
:1078100018684269013A0DD38369191C5143C9188C
:10782000890069180439013BF4D30F68BE0B664325
:107830000E60F7E7F8BDC0464F0400200C0300209F
:10784000F0B5284B89B01E68274B04921A68039143
:107850000592264A3168126807900692244A0191DF
:107860001768019B013B01931FD37468019B214959
:1078700063436518ED18079AAD0002935519013C52
:10788000EFD304992868F8F715FC05990B78002BBD
:1078900007D0069A029953181B5DBA6858435043A3
:1078A000001300042860043DE9E70F490F4B3469D9
:1078B0001F680E68013C13D3039AA5005059049920
:1078C000F8F7F8FB3378002B06D0F0213B1989003C
:1078D0005B181B7858438011039A00045051E9E764
:1078E00009B0F0BD0C0300204C1000205010002007
:1078F00010030020FFFFFF3FF0B591B00693724BDD
:107900000D921C68714A666905901268701E002508
:107910000C9140000FA90F95089208180196049544
:107920000199013907914ED3A36907991F1C774329
:10793000674A5943D218D519059A6D0055190D9A01
:1079400002957F008D0052197F4249000A920997E3
:107950000B91013B33D30A9F9D007D590199A76884
:107960002D0C4F43DF190C990137BF007F58ED1BD9
:10797000099FADB2BC46029FAAB2BC440392171C39
:107980000B9A61468F52089A3FB21278974206DDF1
:107990000299029A09888C46AC44614611800A2FEC
:1079A00003DD0788ED19058005E0002F03DA049A4E
:1079B000AD18ADB20495029D023D0295C9E7079F3F
:1079C00002380197ACE7049A002115B2643504DA55
:1079D000169C01232370081C74E0A5693B4C6E4380
:1079E00020683C4F844605983A68760086191160F5
:1079F0000496FF23013D10D3049E6800305E664666
:107A00003778B842F6D9A94200DAE9B2AB4200DDD4
:107A1000EBB2176838181060ECE72F4D2878049007
:107A200000280FD10FAE0020375EBC460227F65F5C
:107A30006046861B0A2E0DDD069901232B700B7004
:107A400004983FE0256816686878864202D2224F83
:107A500000203870069D2878012806D12668126813
:107A60007078824201D200222A701A4F2268386848
:107A7000527804680020944224D9174C227882421C
:107A800020D1114D5CB22868059E82694069059F2E
:107A9000424348B2001BC40F201840101818C0B24F
:107AA00080189B1840005B009C5F3B5E01209C425D
:107AB00008DD8A1882400598D917125ED00F9342CC
:107AC0004841C0B211B0F0BD0C030020541000209A
:107AD000FFFFFF7F10030020400500202D4BF0B575
:107AE0001D682D4B89B01C680490A7690E1C28687E
:107AF000391C0392F8F7DEFA284B1B68DB799840B3
:107B0000002800DC0120EB6803995843F8F720FBBC
:107B100084466069BB005B42421E391C039351439B
:107B20007B005D425343049CC9198900F318611816
:107B30000595069301900024019D013D019515D303
:107B4000069E0A1CA61907963B1C043A013B08D363
:107B5000079D5E00AD5F66466E431568AD1B156000
:107B6000F3E7039E059B8919E418E5E70C4C102305
:107B7000A371FBB220706370A37004206023211CEA
:107B8000049A2371E070FFF7AFFB0023A37109B0E3
:107B9000F0BDC046100300200C0300204C10002054
:107BA00048040020014B18607047C0465C1000205C
:107BB000014B18687047C0465C10002010B5064C99
:107BC0002060808CFFF7F2FB23683C331878FFF7C6
:107BD000F5FB01F00DFB10BD58100020014B18689B
:107BE0007047C04658100020014B18687047C046C7
:107BF00014030020F7B5484C002120680A224030C9
:107C000001F088FF206800210A224A3001F082FF3B
:107C1000206800212822543001F07CFF20680021D8
:107C20000A227C3001F076FF206800210A2286308B
:107C300001F070FF206800210A22903001F06AFFF5
:107C40002068002105229A3001F064FF206800219D
:107C500005229F3001F05EFF20680021B822C0306D
:107C600001F058FF206800217D302822FF3001F00C
:107C700051FF2A4B24681D68EA69296A5000401A9E
:107C800000024900F8F764FA6B6AA96A071CA06051
:107C90005800401A00024900F8F75AFA204BE060F9
:107CA0001B687F0059681E680139013E09024000C7
:107CB00036028619791800966661216105332A1CFF
:107CC000DB7F271CD832261CA8370192AC36D6356C
:107CD000002B06D010880004F8F73AFA386028889C
:107CE00006E028880004F8F733FA019B386018880A
:107CF00000990004F8F72CFA0A4B30601B686421E5
:107D00001A1C4E32343312781878FC345043F8F78A
:107D10001FFA6067F7BDC046140300205C10002006
:107D20000C030020581000200D4B00211A6830B5BC
:107D3000131CB83319600B4B1B681B7C013BDBB277
:107D4000FF2B0BD059000C5A191C4031490025B2A9
:107D50005118002D00DC0024CC80EFE730BDC04678
:107D6000140300200C03002010B502248B78045764
:107D70005AB2944200DD8370CB78032404575AB280
:107D8000944200DAC3700B78002404575AB294422C
:107D900000DD03704B78012141565AB2914200DA5E
:107DA000437010BDF0B58BB00592059C069301326F
:107DB0002301C418089209912589069E2FB20295C5
:107DC000350145192E892368049636B2B8190790F3
:107DD00028687B4370430799C018F8F7B9F96968B8
:107DE00063684E437B4300B207992060F018F8F7B0
:107DF000AFF900B26060201C109904220A3001F033
:107E000047FE049E029FF319238100232B81069FC6
:107E1000059D099EAD00BA00AC46331CB118634401
:107E200008880027DE5F05B2AE4204DA1880C87801
:107E3000D870897899708449069B09680133C86AAB
:107E4000012583420ADA129E9D40311CB7586144D5
:107E50000E683D4035430D600133F1E7129F00236A
:107E6000BB50069E059F291CB140BD40129A029549
:107E7000CE43069FBB421ADA1068014214D0059D1A
:107E8000AB4203DA029F384310600AE0059DAB4223
:107E900007DD129F381C6044056801279F402F436F
:107EA000076010683040106001330432E1E7109D34
:107EB0002D786DB20295109D0123EB56029E9E42D5
:107EC00000DD9BE0109EB67876B20396109E0322EA
:107ED000029BB256039F0133974200DD8CE05A4A61
:107EE000039D1168119E8F68C96A7B4301335B193A
:107EF000F61832780497013AB4460791531A012BC9
:107F000076DD0121052349420020013B002B29D0C9
:107F10004E4F0126FD187642AE57029DFF18AE194E
:107F2000049D01367543FF790995119E039D7FB22B
:107F300000977719099D7E19009FF6197578013D04
:107F4000E3D3079EB542E0DA059FBD4202D0069E0C
:107F5000B542DAD14F1C03D0A942D6D00120D4E7D4
:107F6000291CD2E7002843D02A2A3FD1089D604629
:107F700005700527013F002F3AD0344B0721DA194D
:107F8000131C5156012252429A562F4B029D1868DB
:107F9000AA188068531C4343039E01337118119E35
:107FA0005B18F0180578002DE4D1139D5B005B5B36
:107FB000002BDFD02A250570258920682EB2594371
:107FC00070430902401861685A435D194E43ADB2CF
:107FD00025812DB21202291CB618F8F7B9F8291C10
:107FE0002060301CF8F7B4F86060C3E763461A708D
:107FF000039D0135039569E702935CE70022AA56C9
:10800000109C0123E3569A421BDC109F0223FB566F
:10801000109F03203856511C834210DC0A48119CE3
:108020000068069D806841430131C91861180878CD
:108030000138A84201D1089E0E700133E8E70A1CFE
:10804000DEE70BB0F0BDC0460C030020FC9F000033
:10805000F0B5A7B02C9C179100940B9213930A9043
:10806000FBF7E4FEC54B1A68131CB4331968C44B04
:10807000012908D1B0321268012A04DD1B689D88ED
:108080001495DB8803E01B681E8814965B881593A3
:10809000BC4B1B68DB6A013B0693069B069E013BBB
:1080A000002E00D172E1139F9A00069CD2590794CA
:1080B000E2400E9206930E9C002CEED0B14B079D31
:1080C0001B68DB6A9D42E8DA0E9D0122154200D151
:1080D0004DE1069E0A9F3501079E7D1934013C192A
:1080E00020682F686E68391A6768F31BCF17CE199E
:1080F0007E40DF170F96DE197E400F9F0C96B74229
:1081000002DD1092180203E0002608021096191CE6
:10811000F8F71EF81CAE211C042212900A31301C04
:1081200001F0B6FC291C0A31301CFFF71DFE28683F
:1081300020900821675E08972768089B0997082107
:108140006F5E5843099B089A7B43BA18111CC018EC
:108150000D92F7F7FDFF21900998646822906868F6
:10816000089D3B1C6343239068430D99C018F7F7A3
:10817000EFFF0027249000211DA80C22259401F078
:10818000C9FCF757012409973457022518947557ED
:108190007C4B1995F6781B6876B21A960D93099E5A
:1081A000189FBE4200DDA0E0099E199F3602169678
:1081B0000897099B089C1A9D0133AC4200DD92E0B0
:1081C0000D98089C80680B9E434301331D190D9F39
:1081D000735DF96A013B11908B4246DB002401205C
:1081E00005224042A446013A002A2DD0664EB71817
:1081F000013F3F78099E7FB2F719119E01377743FF
:108200000597614FBE18F679089F76B204960B9ECB
:10821000F619059FF619049FF6191B967678013E0C
:10822000E1D38E42DFDA069FBE4202D0079FBE42F4
:1082300006D1471C06D0B042D5D00126B446D2E7BD
:108240000124D0E7301CCEE7013049D067466A00F0
:10825000002F01D1002C02D12C9CA05A10E02C9DA3
:10826000591AA85AF7F774FF0AE0002B38DB069E6C
:10827000B34202D0079FBB4232D12C9C6B00185BEB
:1082800000282DD0089D03232902013B28D3109FED
:1082900020AC23AA9E00002F09D09559169FA25901
:1082A0007D1B129F7D432D12551B6D1A08E0A559A9
:1082B000129C4D1B654392592D12169E551BAD1BEA
:1082C000EF17ED197D40FF2DDFDC80267600751B52
:1082D00045439C001DAAA6582D127519A550D4E738
:1082E000089F013764E7099359E71F9B1D9C9C4237
:1082F00000DD1C1C109D002D04D10C9E2B1C002E9B
:108300000FD003E00F9B0C9F0C930F970F9D0C99C0
:10831000A801F7F71DFF3F2800DD3F201A4B181872
:10832000037C2D21149E159FC81A70437B43C018EF
:10833000F7F70EFF44431E9BA412A34217DD079CD0
:10834000069DAC4201DB079506940B9E139F2C9C67
:108350001CAB00930196069B029703940A98179909
:10836000079AFFF71FFD069B079D07930695079E3B
:108370000E9F01367F0807960E979CE61403002097
:10838000581000200C030020FC9F0000404C0121ED
:1083900020684942031CB0331E603E4B18301B68F6
:1083A000DA6A01F0B7FB069E351C3A4F3B68DB6A80
:1083B0009D4226DA0A982F01C71908217B5E002BFF
:1083C0001CDD23681A1CB03211685B190131116081
:1083D0001E76AE4210D00A9A3B68796830011018B8
:1083E000416003603B89391C03810A310A30042251
:1083F00001F04EFB00233B810136F6B20135EDB2B0
:10840000D3E7206800217D302822FF3001F082FB75
:108410003B6822681D680692002158680790A942AF
:108420001CDA0022079F4E1CBA4215DA9868704386
:108430000B9EB7183E187778013F092F0AD8069887
:10844000BF00BE26C7197600B8598446012084446F
:108450006046B8510132E5E7311CDEE722680620AC
:10846000111CB0310C68D221490054500A49079AB6
:108470000B9C4A709A6801238A700132CB70A21853
:1084800030230D700B71FEF72FFF27B0F0BDC046F3
:10849000140300200C03002048040020164BC217D0
:1084A0001B68801850401A1CA83270B5AC33146891
:1084B000CA1789181D68514044434D4324142D1494
:1084C000AC4202DB231C2C1C1D1CA001291CF7F74D
:1084D0003FFE0A4E3018037C281C002B0BD05A227A
:1084E000D21A52365200955B5B0068439D5B0014C4
:1084F0006C432414001970BD14030020FC9F00007D
:10850000F0B58DB000AF7B607E4BFA601D683961BD
:10851000EA6A6946D31DDB08DB00C91A8D466C4642
:108520007C625400231C0833DB08DB00C91A8D462B
:1085300039620121B8614942786A01F0EBFA386A80
:10854000FF21221C01F0E6FA6F4B00261B68FB613D
:108550002C6AA64257DAFC68F300E31804215B5E3C
:10856000002B4DD0331CFC6914339B00E3185A6870
:10857000231CFC33DB6F5200D318FB62231CB03387
:108580001B687C68BB60B300E318002101247B6199
:108590006442B962BB6AB9688B421DDABA6AB969CA
:1085A0001301CB1808215A5E002A10D07A69196885
:1085B0000020105E081A796902228A5E5968891AB9
:1085C000FFF76CFFFA6A904201DABC6AF862BB6A94
:1085D0000133DBB2BB62DDE7621C11D07B6A1A5744
:1085E0006300013207D0396ACB181A88F96A8A42C7
:1085F00006D9198002E0FA6A396ACA527B6A1E55A6
:10860000731CDEB2A4E700243F4B1B68BB62B0338F
:108610001B689C4222DA796A0E5D73B201331AD06C
:10862000F6B20E207043BB693A692101591810183F
:108630004B680A68438002800B89042283800A31D8
:10864000083001F025FA3A6A1436B96A6300B600B8
:108650009B5A8E1973600134E4B2D5E70024B86ADE
:10866000B0300668B44232DA7E6A335701332BD118
:10867000BE692101711808228B5E002B24D02B6A61
:108680009C46002363451FDAFE68D8003018042298
:10869000805E002815D10E2058433E693018042210
:1086A000865E002E0DD17E6A33550A684B680280C3
:1086B00043800B89042283800A31083001F0E8F9F5
:1086C00002E00133DBB2DDE70134E4B2C7E70023A7
:1086D000EC6A2A6AA3420DDABC6AE1180C7E944265
:1086E00003DA7A6A145D0C7601E0FF220A76013320
:1086F000DBB2EDE7964200DD161CBD4606600DB00C
:10870000F0BDC0460C03002014030020F0B595B066
:10871000041C09910A92FFF767FA744B0B901B68CF
:108720001B6A013B0493049D0E236B43E418271D31
:10873000049C013400D1D6E00026BB5F002B00DC96
:10874000CCE06A4B06211868694B07227956BA5665
:108750001B6800248C460C920E93059406940C9E84
:10876000B44566DC05257D57664604223602BA56B6
:108770000D950F960D9D63460133AA4257DC846820
:10878000511C08916143099DC9186B5CC66AB342CC
:1087900024DD0523013B002B2FD0564DEE18ED189C
:1087A000013D2D78F6796DB255190135654376B2E4
:1087B0000295099D03962E1C039D66447519079624
:1087C000029EAE197578002DE4D00E9E6DB275191B
:1087D000ED7D049E6DB2B542DCD109E0002B0BDDCE
:1087E0000B9D1724EB181C57049E0023B44204D1A0
:1087F0000A9C49000B5B00E00023391F0025495FFC
:108800000F9E069D891BCC170919614059436D18AD
:10881000B91E0026895F12028A1AD11752184A40DF
:108820005343059C0695E4180594089AA2E79C46D4
:1088300095E73B1F1A78BB1E1B78802A02DD80213A
:1088400049008A1A802B02DD80214900CB1AD618F4
:10885000294B301C1B681A1CF4320D331168FF338E
:108860000432FEF71EFE254B041C1B680021785EB7
:108870002422995E9A6B40231B1B00930023FEF772
:10888000FFFD2318059C06985C43059400257C5F3A
:108890005843A501291CF7F75BFC291C0690059895
:1088A000F7F756FC011C0698FFF7F8FD144978808D
:1088B000CA7880B212907F20824304234B70134306
:1088C000802252421343049DCB701220B02310AA81
:1088D0001095119613940B71FEF706FD049E0E3F42
:1088E000013E049624E715B0F0BDC0460C030020FD
:1088F00014030020FC9F00005C1000205810002092
:108900001C010020594BF0B51B6885B05A681D6AE0
:10891000013A120202920E241A686B1E5C43013A5D
:108920001202041900270190039204340097002DCD
:1089300000D181E04E4F3B681A1C50321678012E50
:1089400016D102320020215E128891420EDD54338E
:1089500062881B789A4209D946492672B5230E20AF
:1089600000220B71FEF7C0FC009601E00023237289
:108970003E68331C55331B78012B5AD1331C5833B6
:108980000021625E1B889A4253DD231F0027DA5FB5
:10899000FF2A0ADDA31E00201B5EFF2B05DD029FC0
:1089A000BA4202DC039FBB4243DA304B07271B6805
:1089B000E7570533DA7F05200421BC4606272E4BF6
:1089C00020566156E757002A0ED01A68411A131C28
:1089D000AC331B6809024B436046A832C71B1168C1
:1089E0003F021B1479430DE01A686346DF1B131C1A
:1089F000A8331B68AC32411A3F0210687B4309025E
:108A000041431B1409140A208B4201DB584301E047
:108A10004843191CF7F79CFB56363378984208DD1B
:108A20000123144923720E20B62300220B71FEF796
:108A30005BFC013D0E3C7AE7009F002F13D00B4BEF
:108A40000E221B68019F1B6A5A43BA18013B0AD3C6
:108A5000111C0A390020095E002902DD911E012047
:108A600008700E3AF2E705B0F0BDC0460C030020D6
:108A7000581000204F04002014030020F0B51C4BB8
:108A800085B01B6803911B6ADBB2013BDBB2FF2B95
:108A90002CD0039CD900611804254C5F9D0055190A
:108AA000002C1BD00E245C4304190427E65F002E23
:108AB00014D02688019535B2AC4600254F5F654637
:108AC000ED1B6F10BE19019F3E8064880225495F2F
:108AD00026B2711A49100C197C80D6E70E21594331
:108AE00041180C882C8049886980CEE705B0F0BD1C
:108AF0000C03002070B5124C051C20680A227C3043
:108B0000002101F007F80F4B20681B681A6AD2B2E7
:108B1000013AD2B20023FF2A0AD00E21514369182C
:108B20008B8081180E1C4036483133708B70EFE714
:108B30002268111CB031B4320B60136070BDC046A6
:108B4000140300200C03002070B50C4D002428688D
:108B50000526031CB8331C60321C211C9A3000F01F
:108B6000D9FF2868321C211C9F3000F0D3FF2868F1
:108B7000211C0A22863000F0CDFF70BD14030020B6
:108B80000F4AC378126810B551685CB201398C4243
:108B900001DA0133C370837859B2002901DD013B4A
:108BA00083704378126859B2013A914201DA013375
:108BB000437003785AB2002A01DD013B037010BDF7
:108BC0000C030020F0B5B74D8BB007932B680592CE
:108BD0000C1C5A68B449049018684A709A68059E3B
:108BE0008A70012301320870CB70B2180823062066
:108BF0000B71FEF779FB2B68DB6ADBB2013BDBB262
:108C0000FF2B09D0049F1A01BA187F2191721173AA
:108C1000FF21D1725173F1E7A44B00221B68119D13
:108C20001A600922AA56119D0823EB569A4256DB78
:108C3000119E0B217156119F0A23FB5699424CDB62
:108C4000984B501C1E68B768F66A7843059F013040
:108C500040183D182B78B34204DD3E2B3BD800234F
:108C60002B7038E0002B36D0109D4000405B8F4DBC
:108C7000013B2D682E6801362E60049EDDB22B016B
:108C8000F318061C4E431F68BE191E60061C56438F
:108C90005F68BE195E601E8986191E810C269E576C
:108CA000B14200DA19730D269E57B14200DD5973A7
:108CB0000A269E57B24200DA9A720B269E57B2429B
:108CC00000DDDA72AD0065190026AB5F834202DA7F
:108CD0002880EA70A9700139ADE7013AA3E70026C0
:108CE000049F06966F4E069C3368DB6A9C4200DB4D
:108CF000E0E008203B5E002B00D1DBE0381C0A30AE
:108D00000B24FFF73DFF3C5701940A23FB56019DBE
:108D10009D4200DAC1E00D257D5703950C23FB56DB
:108D2000039E9E4200DAB5E05E4B039C1E68019BE9
:108D3000B06801334343059D01331B19ED182A78B0
:108D400000900295002A02D03F2A00D09FE0109D9B
:108D50005B005C5B002C00D199E0002309930523A4
:108D6000013B002B24D0524A0725D1180A1C4D572D
:108D70000121494251560198009A411801314A4354
:108D80000598039994464218521962445178002973
:108D9000E6D0F26A9142E3DC002209A8855C002D4E
:108DA00001D18154DCE78D42FBD00132D2B2F4E72D
:108DB00009AA9A5CDDB2002A04D00133042BF7D152
:108DC0001D1C01E0002D62D0291C201CF7F7C0F902
:108DD000F16A029E013149193170039E0022464317
:108DE0000096019E464302966B1E9C4609AB9B5C17
:108DF000049E013B1B01F318624513DA1E68241A16
:108E0000B446009E0132B44466461E605E68B446B5
:108E1000029EB44466465E601E89B446844466463B
:108E20001E81E1E7039A1868624382181A60019A6A
:108E30005E686243B2185A601A89A4181C81002324
:108E40002A2924DD634522DA01331A1CAA42F9DA01
:108E500009A8C11801390978105C01390138C9B273
:108E6000C0B20124814208D2079E89007118844053
:108E7000201C0C682043086007E0079E8000301823
:108E80008C40211C0468214301600132DEE7039D10
:108E9000013D42E7019C013C36E7069E1037013652
:108EA00006961FE70C03002048040020140300204E
:108EB000FC9F000000253368DC6AA54205DA049FA8
:108EC0002C013C192789002F16D1154A1549126823
:108ED0001868B03215605A68059C4A709A68012378
:108EE0008A7001320870CB70A2182D2306200B71F6
:108EF000FEF7FAF90BB0F0BD21683FB20802391C49
:108F0000F7F726F962682060391C1002F7F720F99C
:108F10006060201C0A300135FFF732FEEDB2CAE76F
:108F20001403002048040020F0B54D4A4D4B126850
:108F30001B6811793822514391B059182C31041C07
:108F400002A800F0A5FD484B00211B685E681F6861
:108F50000733DB7F013F013EFF1A36023F020191DA
:108F6000414D01992B681A6A914276DA0421625EBA
:108F7000002A6DDD0022A05EFF2817DC0533DB7FB1
:108F8000029903AA002B02D06B462A3301E06B46FC
:108F90001633FEF786FA0021635E00B2013BFF3B09
:108FA000584380110130FF30208019E0301AFF282B
:108FB00016DC0533DB7F029903AA002B01D00DAB31
:108FC00000E008ABFEF76DFA0021625E00B2B21A53
:108FD000013AFF3A5043731EFF3B80111B1A238056
:108FE0000222A05EFF2817DC2B6802990533DB7F85
:108FF00003AA002B01D008AB01E06B462A33FEF731
:1090000050FA0221635E00B2013BFF3B58438011DE
:109010000130FF3060801BE0381AFF2818DC2B6815
:1090200002990533DB7F03AA002B02D06B4616336F
:1090300000E00DABFEF735FA0221625E00B2BA1A0B
:10904000013AFF3A50437B1EFF3B80111B1A63809D
:10905000019A0E340132019282E711B0F0BDC04690
:10906000140300205C1000200C030020F8B5144EFF
:10907000041C33680D1C0633DF7FFEF789F9114BA2
:109080001B68FA331B781840336878405A1DD27F2A
:10909000002A0BD02288298821802A8000280DD020
:1090A0001A680733DB7F013AD31A03E0002805D0A2
:1090B0005B68013B22881B029B1A2380F8BDC046D7
:1090C0000C03002000000020F0B5038887B005AC39
:1090D0002380438869461631051C201C0B80FFF74E
:1090E000C5FF354B1B685A1DD17FDE1D334A81CB2E
:1090F00000290CD01268F37F411E013F9068C91A05
:109100003F02DB01029709021B18D7680BE0791EAA
:109110001268F77F0138C01B9368D2680002FF0114
:1091200009020290BF18264A16683268009200228F
:10913000A05E009AC0185B005043C918F7F708F802
:1091400080B2208003906C46706816340190002233
:10915000A05E019B029AC0197F005843D119F6F70F
:10916000F7FF164B80B21B6820801A790123002A72
:1091700001D1D4363378039E05AA31B2994201DC7D
:10918000138007E0009FFE1AB14203DB391C01394E
:10919000C91A118000B2984206DD019EF11A884278
:1091A00003DB311C0139CB1A238013882B802388E1
:1091B0006B8007B0F0BDC0460C03002014030020F4
:1091C0005C100020024B1B68B03318687047C04623
:1091D0001403002038B5041C081C002A07D0D1183D
:1091E000584362434D1010184019F6F7B1FF38BDCF
:1091F00010B5F7F777F9054B01781C68044BFC3480
:109200001B68D868F6F756FFE06710BD140300200E
:1092100058100020F0B5884B0C1C1B6809791B689E
:10922000071C151CFA20627985B08000009150431C
:10923000191C01930392F6F78BFF804B1B68B03328
:109240001A68002A19DD0126B24217D17C4B1B682F
:109250001A6A013A0FD30E235343FB1804215B5EB5
:10926000002BF6DD774901260968E03109888B4239
:1092700008DB321C05E0012604E00026023A531EFA
:109280009A4152420E235343FF183B8802937F8832
:10929000022D18D004D8002D0AD0012D0DD0C3E026
:1092A000052D3ED0062D5CD0042D00D0BCE035E06D
:1092B000002A6BDA012E3CD1B8E0002A6FDA012EC9
:1092C00000D0A5E0B2E0002A09DB5F4B1A78042346
:1092D000002A00D0ADE0009D4F2D60D9A9E0009993
:1092E000FA20800048430199F6F732FF554B1A687F
:1092F000131CE2331B88984207DDE3889C46131C4D
:10930000DC33198803238C4505D8E4321288002306
:10931000904200DA0523012E32D187E0012E08D1D8
:1093200086E0002E07D1474B1B68E4331B88984228
:109330006EDB08237DE0002AFBDB2368029D002111
:109340005A5E28B2801A02229B5E3FB2F91AFFF7DA
:10935000A5F83C4B1B68DE331B789842E9DC002300
:109360005FE00723002E64D00423002A61DB354A26
:109370001268E432128890425BDA6379013350E07C
:10938000022B0CD0052B43D0012B52D12368029D18
:109390005F801D80002201232371E28049E0009D4F
:1093A0002368AA00029DD552227992009A1857800C
:1093B000217989005A1804395B180021505E002574
:1093C000595F401A0225515F02229B5EC91AC317DA
:1093D000C2185A401C4B1D2A08DCCD174A196A4096
:1093E0001D2A03DC5A6801325A6002E000225A60EA
:1093F0001A705A68142A01DD01221A70E588FFF7F5
:109400004DF823792D1801332371E580022310E0F4
:10941000013D0023012D01D9039B01336371052315
:1094200007E06371062304E0002302E0042300E068
:109430002B1C181C05B0F0BD0000002014030020F8
:109440000C0300205C100020EC060020F7B5141C73
:109450000422061C0D1C019300F01AFB0198324AED
:10946000371C8118890070180422691800F010FB5D
:1094700001230093019B0098013B04350437984277
:109480001CDA2B1F0022985E0022AB5E0321C0185D
:109490000422AB5EC018F6F75BFEAB1E38800022DC
:1094A000985E0222AB5E0321C0180622AB5EC01894
:1094B000F6F74EFE009B78800133DAE773880025CB
:1094C000E380A3803388012763802380019A974239
:1094D00027DA0022B35E0422B05EC01A0623F15ED2
:1094E0000222B35EC91AFEF7D9FFB3882D180220F5
:1094F000215E1AB2914200DA63800020215E91421F
:1095000000DD2380F3880622A15E1AB2914200DAC0
:10951000E3800420215E914200DDA3800137043600
:10952000D4E7281CFEBDC046FFFFFF3FF0B58BB05F
:1095300005900391101C15210893F6F709FE0124EC
:10954000069003990598042200F0A2FA00270194DE
:10955000019B08998B4246DA0199039A8B00039983
:10956000D218043B0292CD1800216B5E0020105EE1
:10957000029AC01A0221515E0222AB5EC91AFEF79E
:109580008DFF06993B1804908B4227DB0023EA5E8F
:10959000CF1B0792029A02216E5E0220105E049990
:1095A000801B7843F6F7D4FD029930180990079A8A
:1095B0000020085E059B801AA600049978439E1936
:1095C000F6F7C6FD079B0999181880B28BB2738015
:1095D000308001346B802880002302E0019A013240
:1095E00001921F1CB4E7152C0AD1064BCA18039927
:1095F00092008A18059B11885433198052885A802A
:109600000BB0F0BDFFFFFF3FF7B5051C04228B5EDA
:109610000622885E0C1CC01A642358430223C95ECC
:109620000022A35E0026C91AF6F792FD7623021CDB
:109630001A3AFF33071C9A422FD801960222AB5EDA
:1096400064205843391CF6F783FD019B81B2698081
:10965000012B0DDD2B1F00229B5E0022A85E09B2AC
:10966000C01AAB1E00229B5EC91AFEF717FF361800
:10967000019B043501330193162BDFD10422A05E38
:109680006425391C6843F6F763FDA0800623E05E7D
:10969000391C6843F6F75CFDE080301CFEBDF0B578
:1096A00093B00090151C01930C1C0421565E0622F9
:1096B000AF5E0321BF1B381CF6F74AFD231C503355
:1096C00002215A5E811901248A4200DC00244100F3
:1096D0008E19E4B2B24201DD0222144300229B5EE5
:1096E0000026AA5F8018834201DD042004438A1803
:1096F000934201DD08231C43402202A8002100F010
:1097000009FA0323039306230593012306930423F5
:1097100007930723099302230E9305230F93A400B5
:10972000082311936946E4186358009E391C73702E
:109730000020FEF7B3FE019E011C0A207043F6F7DD
:1097400007FD009E307013B0F0BD0000F0B593B07F
:1097500001900F1C0D1C0126152E0BD13B1C503304
:109760000020195E00203A5E8A1A0220195E02204B
:109770003B5E08E000202B5E04216A5ED21A0623BD
:10978000E95E02202B5ECB1AA821FF315143012450
:1097900089128B4200DC0024194842439212934202
:1097A00001DD022004435242934201DA04221443B1
:1097B00049428B4201DA08231C430021402202A8BF
:1097C00000F0A8F9012302930223039303230593D6
:1097D0000423099308230A9307230E930623109367
:1097E00001990523A4001193083468468B19225867
:1097F000013B01361A700435162EADD113B0F0BD01
:10980000A709000070B5F0B0051C20AC037902AACE
:10981000201C2968FFF71AFE244E021C3368DC3333
:109820001B88984201DC00203EE02B79211C0AA80D
:10983000FFF77CFE02A90AA8FFF7E6FE02AA031CB6
:109840000AA901A8FFF72BFF0AA904A8FFF77EFFCA
:109850000021605E0021FEF721FE0222A15E85B29A
:109860000020FEF71BFE33681A1CE6320024115F4D
:109870002AB29142D7DC191CEA310024095F9142D7
:10988000D1DB1A1CE8320021525E00B28242CADCEF
:10989000EC3300229B5E8342C5DB68460330002325
:1098A00004A90370FAF7F0FF70B070BD5C100020DF
:1098B000014B18607047C04660100020014B1868CB
:1098C0007047C04618030020004870470408000095
:1098D000024B186887239B00C018704718030020AC
:1098E000CE235B005843CC239B00C018014B1B6860
:1098F0001818704718030020024B5843024BC01839
:109900007047C046C503000014B400000A23584342
:10991000C4239B00C018024B1B6818187047C04630
:109920001803002038B5FAF7DBFF0F4B41791B68AD
:10993000012559604279941C2A40A2189A608279C4
:109940001A604A43DA60427902219A61AA40DA61D8
:10995000026859611A62C2791A6101795A1DD17778
:1099600002790633DA7738BD0C03002010B5134CAA
:109970001349144A206800F08BF82068FAF7AAFF10
:109980002068B430F6F79CFD2068F030FDF7A2FDAA
:109990002068F830FEF706F9206886239B00C0187F
:1099A000FDF760FAFFF7BEFF074C201CFAF7AAFF8D
:1099B000064BE018FDF7A6FD10BDC04618030020B9
:1099C00010AC00000408000014B400008A07000076
:1099D00038B5174BCE24596864000A781B68544385
:1099E000CC229200A4181C19124B201C1C60FAF700
:1099F0007DFFC4235B00E518281CFFF759FF201CDE
:109A0000F430F6F769FD862149006018FDF76EFD18
:109A100090225200A018FEF7D1F8281CFDF728FA72
:109A2000054B9A341B6822780733DA7738BDC04675
:109A300018030020641000200C030020014B5B6819
:109A40001870704718030020014B5B681878704746
:109A500018030020F8B50D1C041C081C111C161C52
:109A6000F6F776FB311C071C281CF6F7C7FB002D08
:109A700005DB002908DB2760201C6160F8BD002998
:109A8000F9DD013F8919F6E70137891BF3E7C04685
:109A9000F0B50F2A35D9031C0B439C0735D1161C92
:109AA000103E36093501451910350C1C031C27687A
:109AB0001F6067685F60A7689F60E7681034DF60B9
:109AC0001033AB42F3D1731C1B01C518C9180F2307
:109AD0001340032B1BD91C1FA4080134A40000232E
:109AE000CE58EE500433A342FAD1ED18C91803231F
:109AF0001A4005D00023CC5CEC5401339342FAD1D8
:109B0000F0BD051C002AF5D1FAE7051CF2E71A1C86
:109B1000F8E7C046F0B5830746D0541E002A42D06D
:109B2000CEB2031C032503E0621E002C3BD0141CA4
:109B300001335A1E16702B42F6D1032C2BD9FF2568
:109B40000D402A0215432A0415430F2C15D9271C52
:109B5000103F3F091E1C3A011036B6181A1C15603A
:109B600055609560D5601032B242F8D101373F019F
:109B70000F22DB191440032C0DD9271FBF08BA0090
:109B80001E1DB6181A1C20C2B242FCD10137BF00FC
:109B90000322DB191440002C05D01C19C9B219701E
:109BA0000133A342FBD1F0BD141C031CC5E7C04622
:109BB0000A000000000A0A00010000201F1E1D1CF0
:109BC0001B1A191817000000000000000000000018
:109BD0000000000000000000000000000000000B7A
:109BE0000A0908070605040302000000000000003F
:109BF0000000000000000000000000000000000065
:109C00000000000000000000000000000037180500
:109C100000BF000F00000000000000000000000076
:109C20000000000000000000000000000000000034
:109C300000000000000000F0000000000000000034
:109C40000000000000000000000000000000000014
:109C500000000000830000004001291808000009EE
:109C60000303000011110F0F100F0F0F0F0F111032
:109C70001010100F0F0F0F0F111111100F0F0F0FEA
:109C80000F0F121111101010100F0F0F1111100FD4
:109C90000F0F0F0F0F0F1111111110100F0F0E0FCB
:109CA000111111110F0F0F0F0F0F111011101010B4
:109CB0000F0F0F0E111111110F0F0F0F0F0F1212A7
:109CC0001111101010101010000000000000000012
:109CD0000000000000000000000000000000000084
:109CE0000000000000000000000000000000000074
:109CF0000000000000000000000000000000000064
:109D00000000000000000000000000000000000053
:10A020000000000000000000000000000405AE0178
:10A0300074033B050207CD08940A590C1F0E111139
:10A0400011110F0F0F0F0F0F12121111101010100E
:10A05000101000000600000008000000FF000001D2
:10A06000FF01FF0100FF0100FFFF010100010203EA
:10A07000040405060708090A0B0B0C0D0E0F10113E
:10A0800011121314151516171818191A1B1B1C1D5D
:10A090001D1E1F1F2021212223232424252526279E
:10A0A00027282829292A2A2B2B2C2C2D2D0000008B
:10A0B0007804EF08660DDB115016C21A331FA12376
:10A0C0000C28742CD93039359639EE3D42429046F1
:10A0D000D94A1B4F58538E57BE5BE65F07641F6813
:10A0E000306C397038742F781C7CFF7FD983A88737
:10A0F0006D8B278FD5927996109A9B9D1BA18DA46D
:10A10000F3A74BAB97AED4B104B526B839BB3EBE6E
:10A1100034C11BC4F2C6BAC973CC1BCFB3D13BD474
:10A12000B2D619D96EDBB3DDE6DF08E218E416E635
:10A1300003E8DDE9A5EB5BEDFEEE8FF00DF277F3C2
:10A14000CFF414F646F764F86FF967FA4BFB1BFC83
:10A15000D8FC81FD17FE98FE06FF5FFFA5FFD7FF25
:10A16000F5FFFFFF0400002000000000FF000000DA
:10A1700000000000000000000000000000000000DF
:10A1800000000000000000000000000000000000CF
:10A1900000000000000000000000000000000000BF
:10A1A00000000000000000000000000000000000AF
:10A1B000000000000000000000000000000000009F
:10A1C000000000000000000000000000000000008F
:10A1D000000000000000000000000000000000007F
:10A1E000000000000000000002000000000000006D
:10A1F0001E00000000000000000000000000000041
:10A20000000000000000000000000000000000004E
:10A21000000000000000000000000000000000003E
:10A22000000000000000000000000000000000002E
:10A23000000000000000000000000000000000001E
:10A24000000000000000000000000000030000000B
:10A2500000000000000000000000000000000000FE
:10A2600000000000000000000000000000000000EE
:10A270000000000000000000380300205604002009
:10A280000100000000000001030084000000000045
:10A29000E30400200000000000000000D7040020BC
:10A2A000FF020020F3020020F1020020E002002063
:10A2B00058040020EC010020680400200200000087
:10A2C000D0040020CF0400207A0400200700000002
:10A2D00078040020CF020020CD0200200000000002
:10A2E000C5020020790400200000000000000000EA
:10A2F0000000000000000000A00200208C020020EE
:10A3000000000000000000000000000078020020B3
:10A310000000000064020020000000004C02002049
:10A3200000000000300200200000000000000000DB
:10A33000000000001802002004020020F0010020AC
:10A34000C1020020BC0200200000000073040020B5
:10A3500000200060E80100207004002000020020BE
:10A3600001000000050000006C01002071040020C5
:10A37000140200200100000001000000DC010020A8
:10A380002B02002028020020030000000405070023
:10A39000102000007C010020450200204002002027
:10A3A0000500000008010601040010203031000003
:10A3B000700100205F0200205C020020030000000A
:10A3C0000802060010200000D802002072040020BD
:10A3D000740200200100000004000000440100207D
:10A3E0008A020020880200200200000002110010F2
:10A3F0005C0100209C020020680100200300000096
:10A40000001011002C010020B6020020B002002034
:10A41000060000001708080C0A0C0020304050709D
:10A42000010000000000200601002001021E0001C2
:10A4300000FF00002001027E00000000DC0200207E
:10A4400000600901000100000000000000000000A1
:10A4500000000000000500004D3448504D4500004C
:10A460000000004D49500000000000000400000002
:10A47000000500203005002044050020F8060020DB
:10A48000F4060020FFFFFFFFFFFFFFFFFFFFFFFFBE
:10A49000FFFFFFFFFFFFFFFFFFFFFFFFFFFFFFFFCC
:10A4A000FFFFFFFFFFFFFFFFFFFFFFFFFFFFFFFFBC
:10A4B000FFFFFFFFFFFFFFFFFFFFFFFFFFFFFFFFAC
:10A4C000FFFFFFFFFFFFFFFFFFFFFFFFFFFFFFFF9C
:10AC5000FFFFFFFFFFFFFFFFFFFFFFFFFFFF1501EC
:10AC60004D34485050415241303030303030303027
:10AC70000A000000011F12000100002728292A2BCA
:10AC80002C2D2E2F30313233351211100F0E0D0CAA
:10AC90000B0A09080706050403020000000000244F
:10ACA000232221201F1E1D1C1B1A191817161514EC
:10ACB0001300000000000000000000000000000081
:10ACC0000000000000000000000000000037180530
:10ACD00000BF000F000000000000000000000000A6
:10ACE0000000000000000000000000000000000064
:10ACF00000000000000000F0000000000000000064
:10AD00000000000000000000000000000000000043
:10AD1000000000008000000040032B18080000091C
:10AD200003030000413900000000000000000000A3
:10AD3000000000000A6E6E000100FFFFFFFFFFFF32
:10AD4000FFFFFFFF0A051801E8035000A0006E0096
:10AD50000005641E1E1410143C000000000080005A
:10AD60000A1E3C000080000038040000800700003C
:10AD70000000000038040000000000008007000010
:10AD8000640000000100000001000000010000005C
:10AD9000010000000500000000001000200040003D
:10ADA000800078006E005F0050004B0078006E005D
:10ADB0005F0050004B0078006E005F0050004B00B9
:10ADC0006E006400550046004100000002000000D3
:10ADD000000040008000C400FF005500400000005B
:10ADE0000000000055004000000000000000550079
:10ADF000400000000000000055004000000000007E
:10AE00000000000002000000000040008000C400BC
:10AE1000FF00800080000000000000008000800033
:10AE20000000000000008000800000000000000022
:10AE30008000800000000000000000000505E9021D
:10AE40002D053C00C8000A00D0073200881382009C
:10AE50009001670276022C019001010007000000BA
:10AE600000001900320064009600C800FA000000DB
:10AE70000000000037002D00230019001600140008
:10AE8000120000000000000001000000003F000F61
:10AE900000000000000000000000000000000000B2
:10AEA00000000000000000000000000000000000A2
:10AEB000000000F0000000000000000000000000A2
:10AEC0000000000000000000000000000000000082
:10AED000009E000F000000000000000000000000C5
:10AEE0000000000000000000000000000000000062
:10AEF00000000000000000F0000000000000000062
:10AF00000000000000000000000000000000000041
:10AF1000000000008000000040032B18D1000071E9
:10AF20000A48F61C010000371805371800371805C5
:10AF30000000000000000000000000000000000011
:10AF40000000000000000000000000000000000001
:10AF500000000000000000000000000000000000F1
:10AF600000000000000000000000000000000000E1
:10AF700000000000000000000000000000000000D1
:10AF80000000FFFF0A14380703000000FFFF0A1447
:10AF9000380703000000FFFF0A1438070300000011
:10AFA00000BF010F000000000000000000000000D2
:10AFB0000000000000000000000000000000000091
:10AFC00000000000000000F0000000000000000091
:10AFD0000000000000000000000000000000000071
:10AFE00000000000009E000F0000000000000000B4
:10AFF0000000000000000000000000000000000051
:10B000000000000000000000000000F00000000050
:10B010000000000000000000000000000000000030
:10B0200000000000000000008000000040032B181A
:10B03000D10000710A48F61C0100003718053718C6
:10B0400000371805000000000000000000000000AC
:10B0500000000000000000000000000000000000F0
:10B0600000000000000000000000000000000000E0
:10B0700000000000000000000000000000000000D0
:10B0800000000000000000000000000000000000C0
:10B0900000000000821E96000A0000000700000069
:10B0A000FF7F0080FF7F0080D8FF00000103920235
:10B0B00000005A030800008008070F090CF4400044
:10B0C000B003520326025E0130000000102700008A
:10B0D0000400000000001E002800500000000000D6
:10B0E00000000000280028009600960000000000E4
:10B0F000000000004BA00000C30000001E0F020172
:10B1000002020000070000000F000000010114000F
:10B110000100E80364001900FA000613133D8002E1
:10B1200000012D00780000000100060D28005A00E3
:10B130001414141400002C01E803100000BF020FC7
:10B1400000000000000000000000000000000000FF
:10B1500000000000000000000000000000000000EF
:10B16000000000F0000000000000000000000000EF
:10B1700000000000000000000000000000000000CF
:10B18000009E000F00000000000000000000000012
:10B1900000000000000000000000000000000000AF
:10B1A00000000000000000F00000000000000000AF
:10B1B000000000000000000000000000000000008F
:10B1C000000000008000000040032B18D100007137
:10B1D0000A48F61C01000037180537180037180513
:10B1E000000000000000000000000000000000005F
:10B1F000000000000000000000000000000000004F
:10B20000000000000000000000000000000000003E
:10B21000000000000000000000000000000000002E
:10B22000000000000000000000000000000000001E
:10B23000641E6E000A00000007000000FF7F00800F
:10B24000FF7F0080D8FF00000103920200005A0334
:10B250000800008008070F090CF440008402260251
:10B26000FA00320030000000102700000400000047
:10B2700000001E0028005000000000000000000038
:10B280002800280096009600000000000000000042
:10B290004BA00000C30000001E0F020202020000CB
:10B2A000070000000F000000010114000100E80386
:10B2B00064001900FA000613133D800200012D00FE
:10B2C000780000000100060D28005A00142D142DEE
:10B2D00000002C01E803100000BF000D000000007A
:10B2E000000000000000000000000000000000005E
:10B2F000000000000000000000000000000000F05E
:10B30000000000000000000000000000000000003D
:10B31000000000000000000000000000009E000F80
:10B32000000000000000000000000000000000001D
:10B33000000000000000000000000000000000000D
:10B34000000000F00000000000000000000000000D
:10B3500000000000000000000000000000000000ED
:10B36000400000004003331ED10000710A48F61A65
:10B3700000000137180537180037180500000000D5
:10B3800000000000000000000000000000000000BD
:10B3900000000000000000000000000000000000AD
:10B3A000000000000000000000000000000000009D
:10B3B000000000000000000000000000000000008D
:10B3C000000000000000000000000000641E960065
:10B3D0001400000007000000FF7F0080FF7F008056
:10B3E000D8FF0000010300000000460308000080B1
:10B3F00007070F0A0FF640009D008D005B003A0022
:10B40000300000001027000007000000000032009C
:10B4100000000000000000000000000019001900FA
:10B420000000000000000000000000004BA0000031
:10B43000900100001E0F0201020200000700000040
:10B440000F00000001021400000008076900190045
:10B45000FA000619133D800200012A008000000056
:10B4600000000A0D28005A002D5F010101002C0187
:10B47000E8031000080909090A0B0B0B0C0D0D0D50
:10B480000E0E0F0F0F0F100F100F100E0F0F1010CA
:10B490000F1011080909090A0B0B0B0C0D0D0D0EED
:10B4A0000E0E0F0F0E0F0E0F0E0F0E100E0F0E0FB3
:10B4B0000E100808090A0A0A0B0C0C0C0D0D0D0ED3
:10B4C0000E0E0F0F0F0E0F100F0E0F0E100F100F8E
:10B4D0000F080809090A0A0B0B0C0C0C0D0D0E0EB7
:10B4E0000E0F0E0F0E0F0F0F0F0F0F0F0F0F0F0F6F
:10B4F000080809090A0A0A0B0B0C0C0D0D0D0D0D9D
:10B500000E0F0F0D0F0E0F0E0F0E0F0E0E0E0F085B
:10B51000080909090A0A0B0B0C0C0C0D0D0E0E0E76
:10B520000E0E0E0F0E0F0F0F0E0F0E0E0F0F080840
:10B530000809090A0A0A0B0C0C0C0D0D0E0E0E0E52
:10B540000E0E0E0E0F0F0F0E0E0E0E0E0F0708082A
:10B5500008090A0A0A0B0C0B0C0C0D0D0E0E0D0E31
:10B560000D0E0D0E0E0E0D0E0D0E0F0F0707080916
:10B5700009090A0A0B0B0B0C0C0C0D0D0D0D0E0D11
:10B580000E0E0E0E0E0D0E0D0E0D0D0707080808FF
:10B5900009090A0A0B0B0C0C0C0C0C0E0C0E0D0EF0
:10B5A0000D0D0D0E0D0E0D0D0D0E060707080808EA
:10B5B000090A0A0A0A0B0B0C0C0C0D0D0D0D0D0ED1
:10B5C0000D0E0D0E0E0E0D0E0E06070707080809CC
:10B5D0000909090A0B0A0B0B0B0D0C0D0C0D0C0DB8
:10B5E0000C0D0C0D0D0D0C0E0606070707080809BB
:10B5F00009090A0A0A0B0B0B0C0B0C0C0C0D0D0D98
:10B600000D0D0C0C0C0C0D050606070707080808A5
:10B610000909090A0A0B0B0B0B0B0B0C0C0C0D0C7C
:10B620000C0C0B0C0C0C050606060707080808098D
:10B6300009090A0A0A0A0B0C0B0C0B0C0C0C0C0C5B
:10B640000B0C0C0C0C050506060707070708090973
:10B650000909090A0B0B0B0B0B0C0B0C0B0C0B0C3D
:10B660000B0C0C0D05050606060607070808090859
:10B6700009090A0A0B0A0B0A0B0B0C0B0C0B0B0B20
:10B680000B0B0C0405050606060707070808080942
:10B6900008090A0A0A0A0A0B0B0B0B0B0B0B0B0B04
:10B6A0000B0B000000000000000000000000000084
:10B6B000000000000000000000000000000000008A
:10B6C000000000000000000000000000000000007A
:10B6D000000000000000000000000000000000006A
:10B6E000000000000000000000000000000000005A
:10B6F000000000000000000000000000000000004A
:10B700000000000000000000000000000000000039
:10B710000000000000000000000000000000000029
:10B720000000000000000000000000000000000019
:10B730000000000000000000000000000000000009
:10B7400000000000000000000000000000000000F9
:10B7500000000000000000000000000000000000E9
:10B7600000000000000000000000000000000000D9
:10B7700000000000000000000000000000000000C9
:10B7800000000000000000000000000000000000B9
:10B7900000000000000000000000000000000000A9
:10B7A0000000000000000000000000000000000099
:10B7B0000000000000000000000000000000000089
:10B7C0000000000000000000000000000000000079
:10B7D0000000000000000000000000000000000069
:10B7E0000000000000000000000000000000000059
:10B7F0000000000000000000000000000000000049
:10B800000000000000000000000000000000000038
:10B810000000000000000000000000000000000028
:10B820000000000000000000000000000000000018
:10B83000000000000000000000080909090A0B0BC5
:10B840000B0C0D0D0D0E0E0F0F0F0F100F100F1014
:10B850000E0F0F10100F1011080909090A0B0B0B1E
:10B860000C0D0D0D0E0E0E0F0F0E0F0E0F0E0F0EF8
:10B87000100E0F0E0F0E100808090A0A0A0B0C0C06
:10B880000C0D0D0D0E0E0E0F0F0F0E0F100F0E0FD5
:10B890000E100F100F0F080809090A0A0B0B0C0CE9
:10B8A0000C0D0D0E0E0E0F0E0F0E0F0F0F0F0F0FB4
:10B8B0000F0F0F0F0F080809090A0A0A0B0B0C0CCF
:10B8C0000D0D0D0D0D0E0F0F0D0F0E0F0E0F0E0F98
:10B8D0000E0E0E0F08080909090A0A0B0B0C0C0CB6
:10B8E0000D0D0E0E0E0E0E0E0F0E0F0F0F0E0F0E75
:10B8F0000E0F0F08080809090A0A0A0B0C0C0C0D98
:10B900000D0E0E0E0E0E0E0E0E0F0F0F0E0E0E0E55
:10B910000E0F07080808090A0A0A0B0C0B0C0C0D7D
:10B920000D0E0E0D0E0D0E0D0E0E0E0D0E0D0E0F3C
:10B930000F0707080909090A0A0B0B0B0C0C0C0D61
:10B940000D0D0D0E0D0E0E0E0E0E0D0E0D0E0D0D1F
:10B95000070708080809090A0A0B0B0C0C0C0C0C49
:10B960000E0C0E0D0E0D0D0D0E0D0E0D0D0D0E0609
:10B970000707080808090A0A0A0A0B0B0C0C0C0D29
:10B980000D0D0D0D0E0D0E0D0E0E0E0D0E0E0607ED
:10B9900007070808090909090A0B0A0B0B0B0D0C0C
:10B9A0000D0C0D0C0D0C0D0C0D0D0D0C0E060607DF
:10B9B000070708080909090A0A0A0B0B0B0C0B0CEC
:10B9C0000C0C0D0D0D0D0D0C0C0C0C0D05060607C9
:10B9D00007070808080909090A0A0B0B0B0B0B0BD0
:10B9E0000C0C0C0D0C0C0C0B0C0C0C0506060607B5
:10B9F000070808080909090A0A0A0A0B0C0B0C0BAC
:10BA00000C0C0C0C0C0B0C0C0C0C0505060607079B
:10BA100007070809090909090A0B0B0B0B0B0C0B8B
:10BA20000C0B0C0B0C0B0C0C0D0505060606060783
:10BA3000070808090809090A0A0B0A0B0A0B0B0C6C
:10BA40000B0C0B0B0B0B0B0C04050506060607076E
:10BA5000070808080908090A0A0A0A0A0B0B0B0B4F
:10BA60000B0B0B0B0B0B0B00000000000000000089
:10BA700000000000000000000000000000000000C6
:10BA800000000000000000000000000000000000B6
:10BA900000000000000000000000000000000000A6
:10BAA0000000000000000000000000000000000096
:10BAB0000000000000000000000000000000000086
:10BAC0000000000000000000000000000000000076
:10BAD0000000000000000000000000000000000066
:10BAE0000000000000000000000000000000000056
:10BAF0000000000000000000000000000000000046
:10BB00000000000000000000000000000000000035
:10BB10000000000000000000000000000000000025
:10BB20000000000000000000000000000000000015
:10BB30000000000000000000000000000000000005
:10BB400000000000000000000000000000000000F5
:10BB500000000000000000000000000000000000E5
:10BB600000000000000000000000000000000000D5
:10BB700000000000000000000000000000000000C5
:10BB800000000000000000000000000000000000B5
:10BB900000000000000000000000000000000000A5
:10BBA0000000000000000000000000000000000095
:10BBB0000000000000000000000000000000000085
:10BBC0000000000000000000000000000000000075
:10BBD0000000000000000000000000000000000065
:10BBE0000000000000000000000000000000000055
:10BBF0000000000000000000000000000000191913
:10BC00001B1E2021232627292B2C2E2F2F303133AA
:10BC10003235353635383737383A3A39411716180C
:10BC20001B1C1D1F2122232526282828292B2D2CCB
:10BC30002D2D2E2E2F2F302F303032381717181A67
:10BC40001C1D1F2122232325272828292A2B2B2CA2
:10BC50002C2D2D2F2F2F2E2F2F30391717181A1D5F
:10BC60001D1F2122232324262727292A2B2C2C2D74
:10BC70002D2D2E2E2E2F2E2F30391817191B1C1E4E
:10BC80001F2122232424262727292B2B2B2D2D2E41
:10BC90002D2F2E2F2E2F2F31391717191B1D1E1F39
:10BCA000212324242526282729292A2C2D2D2E2E10
:10BCB0002E2E2F2E2F2F30381717191B1C1E1F2228
:10BCC00023232526272827282A2B2C2C2D2D2D2EE3
:10BCD0002E2E2E2F2F31391717191B1C1D1F212215
:10BCE00023252628282728292B2B2D2D2E2E2E2FB5
:10BCF000302F302F30381717191B1C1E1F212223FD
:10BD00002526272828282A2B2B2C2C2C2D2E2F2F8C
:10BD10002F2F2E30381716181A1C1D1F21222324EE
:10BD200027272727292A2B2B2C2C2D2D2E2E2E2E64
:10BD30002F2F30371616181A1B1D1E2021232526DB
:10BD4000272827282A2A2B2C2C2C2D2D2E2D2E2D42
:10BD50002E3037161517191B1C1E1F2122242627CB
:10BD600028272A2A2A2B2C2B2C2C2D2D2E2E2D2E1B
:10BD70003036151516181A1B1D1F202123252626BF
:10BD8000262829292A2A2B2C2C2C2C2D2D2C2D2F02
:10BD90003615141617191A1C1E20212225262626B0
:10BDA00026282929292A2A2B2C2D2D2D2C2C2E35DD
:10BDB00014141517191A1C1E1F21222425252526A7
:10BDC00028282827292B2B2C2C2D2D2B2C2E3313D8
:10BDD000131517191A1C1D1F212224252526262775
:10BDE000282727272B2B2C2C2D2D2D2C2D311312D2
:10BDF0001416191A1B1D1F21222426252627282840
:10BE00002728292A2C2D2D2D2D2D2D2D31151417B8
:10BE1000191B1D1F212426272A2B2C2C2E2E2E2DBC
:10BE20002F2E3032333333333332313300000000BE
:10BE30000000000000000000000000000000000002
:10BE400000000000000000000000000000000000F2
:10BE500000000000000000000000000000000000E2
:10BE600000000000000000000000000000000000D2
:10BE700000000000000000000000000000000000C2
:10BE800000000000000000000000000000000000B2
:10BE900000000000000000000000000000000000A2
:10BEA0000000000000000000000000000000000092
:10BEB0000000000000000000000000000000000082
:10BEC0000000000000000000000000000000000072
:10BED0000000000000000000000000000000000062
:10BEE0000000000000000000000000000000000052
:10BEF0000000000000000000000000000000000042
:10BF00000000000000000000000000000000000031
:10BF10000000000000000000000000000000000021
:10BF20000000000000000000000000000000000011
:10BF30000000000000000000000000000000000001
:10BF400000000000000000000000000000000000F1
:10BF500000000000000000000000000000000000E1
:10BF600000000000000000000000000000000000D1
:10BF700000000000000000000000000000000000C1
:10BF800000000000000000000000000000000000B1
:10BF900000000000000000000000000000000000A1
:10BFA0000000000000000000000000000000000091
:10BFB0000000000000000000000000000000000081
:10BFC000000000FFFFFFFFFFFFFFFFFFFFFFFFFF7E
:10BFD000FFFFFFFFFFFFFFFFFFFFFFFFFFFFFFFF71
:10BFE000FFFFFFFFFFFFFFFFFFFFFFFFFFFFFFFF61
:10BFF000FFFFFFFFFFFFFFFFFFFFFFFFFFFFFFFF51
:10C00000FFFFFFFFFFFFFFFFFFFFFFFFFFFFFFFF40
:10C01000FFFFFFFFFFFFFFFFFFFFFFFFFFFF150118
:10C020004D4254014D3448500000000000C0000053
:10C03000EEEE110215011501EEEEEEEE002B2B30A7
:10C040000022090100140000040516201148150003
:10C05000000000000000000000004000F039000077
:00000001FF
